:020000040000FA
:1000000002EF00F00F01BF0E926E300E936E000EE5
:10001000946E000E956E0F0E966E030E386F300EB6
:10002000396F000E3A6F000E3B6F000E3C6F010EF1
:10003000C26E040EC16EB20EC06E700ED36E400E54
:100040009B6E806A816A826A836A846A896A8A6A24
:100050008B6A8C6A8D6A00018C8C006A016A026A64
:10006000036A046A056A066A076A086A096A0A6A0C
:100070000B6A0C6A0D6A0E6A0F6A106A116A126ABC
:10008000136A146A156A166A176A186A196A1A6A6C
:100090001B6A1C6A1D6A1E6A1F6A206A216A226A1C
:1000A000236A246A256A266A276A286A296A2A6ACC
:1000B0002B6A2C6A316A326A336A346A356A366A64
:1000C000376A386A396A3A6A3B6A3C6A3D6A3E6A0C
:1000D0003F6A406A416A426A436A446A456A466ABC
:1000E000476A4D6A4E6A4F6A506A516A526A536A49
:1000F000546A556A566A576A586A596A5A6A5B6AF4
:100100005C6A5D6A5E6A5F6A8A82E6EC29F0BEEC30
:100110001AF036EC18F0C00E8B6E8C928C900000AA
:10012000000000000000000000008C8400000000BF
:1001300000000000000000000000000000000000BF
:1001400000000000000000000000000000000000AF
:100150000000000000000000000000008C9400007F
:10016000000000000000000000000000000000008F
:10017000000000000000000000000000000000007F
:10018000B7EC18F03F0E8B6E8C928C900000000044
:1001900000000000000000008C840000000000004F
:1001A000000000000000000000000000000000004F
:1001B000000000000000000000000000000000003F
:1001C000000000000000000000008C94000000000F
:1001D000000000000000000000000000000000001F
:1001E0000000000000000000000000000000A0EC83
:1001F00019F08C8E39EC18F0DEEC1AF0C46AC36A80
:10020000000EAA6E000EA96EA69EA69CA6800000F7
:100210000000A8503F6E000EAA6E010EA96EA69EA9
:10022000A69CA68000000000A8504F6E000EAA6E8B
:10023000020EA96EA69EA69CA68000000000A850F3
:100240005A6E000EAA6E070EA96EA69EA69CA680E8
:1002500000000000A850506E3F504E6E4F50516E3F
:100260005A505B6E3FAC63EF01F0000EAA6E030EB6
:10027000A96EA69EA69CA68000000000A850246E31
:10028000000EAA6E040EA96EA69EA69CA680000073
:100290000000A850256E000EAA6E050EA96EA69E3F
:1002A000A69CA68000000000A850266E000EAA6E34
:1002B000060EA96EA69EA69CA68000000000A8506F
:1002C000276EE6EC29F08C86898C3F9032EC1EF08C
:1002D00012EC27F03FAA70EF01F08A8071EF01F075
:1002E0008A9080B48EEF01F00C0E545CD8B47CEF91
:1002F00001F0542A90EF01F0546A11BA90EF01F026
:10030000118A3FA089EF01F08C86898C3F9090EF95
:1003100001F08C96899C3F8090EF01F0119A546A0D
:1003200084B00AEF02F00C0E575CD8B49BEF01F0DA
:10033000572A0CEF02F0576A11B80CEF02F011883F
:10034000000E145CD8B4B1EF01F0010E145CD8B407
:10035000B3EF01F0020E145CD8B4D1EF01F0E9EF75
:1003600001F00CEF02F012B0C4EF01F0196A12A212
:100370001A6A12A41B6A146A446A456A466A476A82
:10038000A0EC19F00CEF02F03F504E6E1C6A196A97
:100390001290446A456A466A476AA0EC19F00CEF6D
:1003A00002F012B2E2EF01F01A6A12A0196A12A466
:1003B0001B6A146A446A456A466A476AA0EC19F0E7
:1003C0000CEF02F04F50516E5A505B6E12920CEFD0
:1003D00002F012B4FAEF01F01B6A12A0196A12A21D
:1003E0001A6A146A446A456A466A476AA0EC19F0B8
:1003F0000CEF02F0539053923FAC02EF02F04E8CA0
:1004000003EF02F04E9CA0EC19F01B6A12941E9EA2
:100410000CEF02F01198576A84B2C0EF02F00C0E94
:10042000585CD8B417EF02F0582AC2EF02F0586AAD
:1004300011B6C2EF02F01186000E145CD8B42DEF95
:1004400002F0010E145CD8B446EF02F0020E145C08
:10045000D8B458EF02F073EF02F0406A416A426A82
:10046000436A446A456A466A476A316A326A336A4D
:10047000346A356A366A376A386A50A043EF02F048
:100480005090C2EF02F05080C2EF02F012B04CEF79
:1004900002F01280C2EF02F03FA052EF02F04E8055
:1004A00053EF02F04E904E503F6E1290C2EF02F0AA
:1004B00012B25EEF02F01282C2EF02F051504F6EA4
:1004C0005B505A6E316A326A336A346A356A366A08
:1004D000376A386A396A3A6A3B6A3C6A3D6A3E6AF8
:1004E0001292C2EF02F012B479EF02F01284C2EF5E
:1004F00002F0000E1B5CD8A498EF02F053A095EF19
:1005000002F053909EEC31F0B2EC31F0C5EC31F0DA
:1005100024EC32F03FAC95EF02F0D8EC31F0EBEC8C
:1005200031F0FEEC31F011EC32F01294C2EF02F037
:10053000020E1B5CD8A4B6EF02F053A2B3EF02F098
:1005400053923F6A4E6A3F8A4E8A8C86898C4F6AE4
:10055000516A010E5A6E010E5B6E246A256A266A84
:10056000276AE6EC29F01294C2EF02F04EACBCEF21
:1005700002F03F8CBDEF02F03F9C1294C2EF02F0FC
:100580001196586A84B4E5EF02F00C0E595CD8B4A9
:10059000CDEF02F0592AE7EF02F0596A11B0E7EF08
:1005A00002F01180030E145CD8B4DCEF02F0142AC0
:1005B000A0EC19F0E7EF02F0146A446A456A466A53
:1005C000476AA0EC19F0E7EF02F01190596A000EAB
:1005D000145CD8B4F8EF02F0010E145CD8B495EFB7
:1005E0000AF0020E145CD8B4BAEF0EF0C5EF13F0A7
:1005F00012EC27F030EC18F0410E3CEC18F0B80E7D
:1006000064EC18F0700E8CEC18F0100E8CEC18F0F6
:10061000100E8CEC18F0100E8CEC18F0000E8CEC18
:1006200018F0D8EC2EF0000E8CEC18F068EC2EF0E0
:10063000000E8CEC18F038EC2EF0000E8CEC18F05C
:10064000C8EC2EF0000E8CEC18F048EC2EF0000EEA
:100650008CEC18F0D8EC2DF008EC31F0A8EC2EF072
:10066000000E8CEC18F0B8EC2EF0000E8CEC18F0AC
:1006700098EC2DF033EC18F0400E3CEC18F0B80E6E
:1006800064EC18F0B8EC2EF0000E8CEC18F0C8EC0E
:100690002EF0000E8CEC18F0A8EC2EF0000E8CEC76
:1006A00018F0082A2D0E085CD8B45CEF03F0100E89
:1006B0008CEC18F051EF03F0086A700E8CEC18F017
:1006C00030EC18F0410E3CEC18F0BB0E64EC18F066
:1006D000700E8CEC18F0100E8CEC18F0100E8CECE8
:1006E00018F0100E8CEC18F0000E8CEC18F038ECB2
:1006F0002EF008EC31F0B8EC2DF0000E8CEC18F078
:1007000008EC2EF0000E8CEC18F0082A230E085C82
:10071000D8B490EF03F0100E8CEC18F085EF03F0D6
:10072000086A700E8CEC18F033EC18F0410E3CECBB
:1007300018F0BB0E64EC18F0700E8CEC18F0100E74
:100740008CEC18F0100E8CEC18F0100E8CEC18F0ED
:10075000000E8CEC18F098EC2EF008EC31F0B8ECB0
:100760002DF0000E8CEC18F008EC2EF0000E8CEC46
:1007700018F0082A230E085CD8B4C4EF03F0100E5A
:100780008CEC18F0B9EF03F0086A700E8CEC18F0DE
:1007900012EC27F030EC18F0410E3CEC18F0BC0ED7
:1007A00064EC18F038EC2EF0000E8CEC18F078ECBD
:1007B0002EF0000E8CEC18F02CEC31F0000E8CECCE
:1007C00018F0000E8CEC18F02450286E000E285CF7
:1007D000D8A40AEF04F0000E8CEC18F008EC31F00D
:1007E000000E8CEC18F04CEC31F0000E8CEC18F094
:1007F0004CEC31F0000E8CEC18F0400E8CEC18F044
:10080000000E8CEC18F04CEC31F0000E8CEC18F073
:10081000A7EF04F0C00E285CD8B416EF04F0C00EA9
:10082000285CD8A035EF04F07DEF04F0000E8CECCE
:1008300018F008EC31F0000E8CEC18F0B8EC2AF04F
:10084000000E8CEC18F0B8EC2AF0000E8CEC18F0CE
:10085000400E8CEC18F0000E8CEC18F0B8EC2AF07E
:10086000000E8CEC18F0A7EF04F04CEC31F0000E09
:100870008CEC18F0000E8CEC18F0BF0E285CD8A49D
:1008800059EF04F0B8EC2AF0000E8CEC18F0B8EC3C
:100890002AF0000E8CEC18F0400E8CEC18F0000ED4
:1008A0008CEC18F008EC2BF0000E8CEC18F0A7EF95
:1008B00004F02450286E281E282A400E285E284264
:1008C000289E285063EC1DF0B5EC1DF0400E8CEC1A
:1008D00018F0000E8CEC18F024A076EF04F008EC71
:1008E0002BF0000E8CEC18F0A7EF04F0B8EC2AF017
:1008F000000E8CEC18F0A7EF04F03CEC31F0000E89
:100900008CEC18F0000E8CEC18F02450286E284265
:10091000289E289C289A285063EC1DF0B5EC1DF009
:10092000400E8CEC18F0000E8CEC18F024A0A0EF18
:1009300004F008EC2BF0000E8CEC18F0A7EF04F09C
:10094000B8EC2AF0000E8CEC18F0A7EF04F0000EC3
:100950008CEC18F038EC2FF0000E8CEC18F0A8ECB2
:100960002DF0000E8CEC18F030EC18F0410E3CEC41
:1009700018F0BD0E64EC18F038EC2EF0000E8CEC84
:1009800018F058EC2EF0000E8CEC18F02CEC31F036
:10099000000E8CEC18F0000E8CEC18F02550286E30
:1009A000000E285CD8A4F4EF04F0000E8CEC18F0D4
:1009B00008EC31F0000E8CEC18F04CEC31F0000E2D
:1009C0008CEC18F04CEC31F0000E8CEC18F0400E72
:1009D0008CEC18F0000E8CEC18F04CEC31F0000EA2
:1009E0008CEC18F091EF05F0C00E285CD8B400EF45
:1009F00005F0C00E285CD8A01FEF05F067EF05F0EA
:100A0000000E8CEC18F008EC31F0000E8CEC18F0B5
:100A1000B8EC2AF0000E8CEC18F0B8EC2AF0000EBE
:100A20008CEC18F0400E8CEC18F0000E8CEC18F0EA
:100A3000B8EC2AF0000E8CEC18F091EF05F04CECBD
:100A400031F0000E8CEC18F0000E8CEC18F0BF0E9C
:100A5000285CD8A443EF05F0B8EC2AF0000E8CEC2B
:100A600018F0B8EC2AF0000E8CEC18F0400E8CEC6C
:100A700018F0000E8CEC18F008EC2BF0000E8CEC4B
:100A800018F091EF05F02550286E281E282A400EF8
:100A9000285E2842289E285063EC1DF0B5EC1DF01E
:100AA000400E8CEC18F0000E8CEC18F025A060EFD6
:100AB00005F008EC2BF0000E8CEC18F091EF05F02F
:100AC000B8EC2AF0000E8CEC18F091EF05F03CEC3D
:100AD00031F0000E8CEC18F0000E8CEC18F0255064
:100AE000286E2842289E289C289A285063EC1DF0E6
:100AF000B5EC1DF0400E8CEC18F0000E8CEC18F0EC
:100B000025A08AEF05F008EC2BF0000E8CEC18F015
:100B100091EF05F0B8EC2AF0000E8CEC18F091EF94
:100B200005F0000E8CEC18F038EC2FF0000E8CEC79
:100B300018F0A8EC2DF0000E8CEC18F012EC27F059
:100B400033EC18F0410E3CEC18F0BC0E64EC18F0DD
:100B500098EC2EF0000E8CEC18F078EC2EF0000ED5
:100B60008CEC18F02CEC31F0000E8CEC18F0000E30
:100B70008CEC18F02650286E000E285CD8A4E0EF0C
:100B800005F0000E8CEC18F008EC31F0000E8CEC47
:100B900018F04CEC31F0000E8CEC18F04CEC31F00D
:100BA000000E8CEC18F0400E8CEC18F0000E8CEC63
:100BB00018F04CEC31F0000E8CEC18F07DEF06F0E4
:100BC000C00E285CD8B4ECEF05F0C00E285CD8A0AD
:100BD0000BEF06F053EF06F0000E8CEC18F008EC6B
:100BE00031F0000E8CEC18F0B8EC2AF0000E8CEC12
:100BF00018F0B8EC2AF0000E8CEC18F0400E8CECDB
:100C000018F0000E8CEC18F0B8EC2AF0000E8CEC0A
:100C100018F07DEF06F04CEC31F0000E8CEC18F083
:100C2000000E8CEC18F0BF0E285CD8A42FEF06F055
:100C3000B8EC2AF0000E8CEC18F0B8EC2AF0000E9C
:100C40008CEC18F0400E8CEC18F0000E8CEC18F0C8
:100C500008EC2BF0000E8CEC18F07DEF06F026501F
:100C6000286E281E282A400E285E2842289E2850DA
:100C700063EC1DF0B5EC1DF0400E8CEC18F0000E8E
:100C80008CEC18F026A04CEF06F008EC2BF0000ED0
:100C90008CEC18F07DEF06F0B8EC2AF0000E8CEC2E
:100CA00018F07DEF06F03CEC31F0000E8CEC18F003
:100CB000000E8CEC18F02650286E2842289E289CA6
:100CC000289A285063EC1DF0B5EC1DF0400E8CEC1A
:100CD00018F0000E8CEC18F026A076EF06F008EC69
:100CE0002BF0000E8CEC18F07DEF06F0B8EC2AF03B
:100CF000000E8CEC18F07DEF06F0000E8CEC18F076
:100D000038EC2FF0000E8CEC18F0A8EC2DF0000E53
:100D10008CEC18F012EC27F033EC18F0410E3CECA0
:100D200018F0BD0E64EC18F098EC2EF0000E8CEC70
:100D300018F058EC2EF0000E8CEC18F02CEC31F082
:100D4000000E8CEC18F0000E8CEC18F02750286E7A
:100D5000000E285CD8A4CCEF06F0000E8CEC18F046
:100D600008EC31F0000E8CEC18F04CEC31F0000E79
:100D70008CEC18F04CEC31F0000E8CEC18F0400EBE
:100D80008CEC18F0000E8CEC18F04CEC31F0000EEE
:100D90008CEC18F069EF07F0C00E285CD8B4D8EFDF
:100DA00006F0C00E285CD8A0F7EF06F03FEF07F082
:100DB000000E8CEC18F008EC31F0000E8CEC18F002
:100DC000B8EC2AF0000E8CEC18F0B8EC2AF0000E0B
:100DD0008CEC18F0400E8CEC18F0000E8CEC18F037
:100DE000B8EC2AF0000E8CEC18F069EF07F04CEC30
:100DF00031F0000E8CEC18F0000E8CEC18F0BF0EE9
:100E0000285CD8A41BEF07F0B8EC2AF0000E8CEC9D
:100E100018F0B8EC2AF0000E8CEC18F0400E8CECB8
:100E200018F0000E8CEC18F008EC2BF0000E8CEC97
:100E300018F069EF07F02750286E281E282A400E68
:100E4000285E2842289E285063EC1DF0B5EC1DF06A
:100E5000400E8CEC18F0000E8CEC18F027A038EF48
:100E600007F008EC2BF0000E8CEC18F069EF07F09F
:100E7000B8EC2AF0000E8CEC18F069EF07F03CECAF
:100E800031F0000E8CEC18F0000E8CEC18F02750AE
:100E9000286E2842289E289C289A285063EC1DF032
:100EA000B5EC1DF0400E8CEC18F0000E8CEC18F038
:100EB00027A062EF07F008EC2BF0000E8CEC18F086
:100EC00069EF07F0B8EC2AF0000E8CEC18F069EF2F
:100ED00007F0000E8CEC18F038EC2FF0000E8CECC4
:100EE00018F0A8EC2DF0000E8CEC18F012EC27F0A6
:100EF00030EC18F0400E3CEC18F0BA0E64EC18F030
:100F00003FA09CEF07F0FF0E8CEC18F018EC30F0CF
:100F1000FF0E8CEC18F098EC30F0FF0E8CEC18F013
:100F200088EC30F0FF0E8CEC18F098EC2FF0FF0EF0
:100F30008CEC18F0B3EF07F0000E8CEC18F008EC16
:100F400031F0000E8CEC18F008EC31F0000E8CEC57
:100F500018F008EC31F0000E8CEC18F008EC31F0D1
:100F6000000E8CEC18F030EC18F0400E3CEC18F051
:100F7000B90E64EC18F03FB218EF08F0FF0E8CECDD
:100F800018F0D8EC2FF0FF0E8CEC18F028EC30F0B5
:100F9000FF0E8CEC18F088EC30F0FF0E8CEC18F0A3
:100FA00098EC2FF0FF0E8CEC18F068EC30F0FF0E90
:100FB0008CEC18F008EC30F0FF0E8CEC18F038ECEC
:100FC00030F0FF0E8CEC18F078EC2FF0FF0E8CEC6C
:100FD00018F0F8EC2FF0FF0E8CEC18F008EC31F064
:100FE000000E8CEC18F0000E8CEC18F0000E8CEC5F
:100FF00018F0000E8CEC18F033EC18F0400E3CECBE
:1010000018F0B90E64EC18F0000E8CEC18F0000E1D
:101010008CEC18F008EC31F0000E08EC31F0000E0A
:1010200008EC31F0000E08EC31F0000ECBEF08F0C8
:10103000FF0E8CEC18F078EC30F0FF0E8CEC18F012
:1010400098EC2FF0FF0E8CEC18F048EC30F0FF0E0F
:101050008CEC18F058EC2FF0FF0E8CEC18F068ECCC
:1010600030F0FF0E8CEC18F058EC2FF0FF0E8CECEB
:1010700018F088EC30F0FF0E8CEC18F098EC2FF0A4
:10108000FF0E8CEC18F018EC31F0FF0E8CEC18F021
:101090003FA452EF08F068EC30F0FF0E8CEC18F033
:1010A00057EF08F008EC30F0FF0E8CEC18F03FB66C
:1010B00087EF08F0000E8CEC18F0000E8CEC18F0A6
:1010C000000E8CEC18F033EC18F0400E3CEC18F0ED
:1010D000B90E64EC18F0000E8CEC18F0000E8CECDD
:1010E00018F008EC31F0000E8CEC18F008EC31F040
:1010F000000E8CEC18F008EC31F0000E8CEC18F0BF
:1011000008EC31F0000E8CEC18F0CBEF08F0FF0E7D
:101110008CEC18F0FF0E8CEC18F0FF0E8CEC18F035
:1011200033EC18F0400E3CEC18F0B90E64EC18F0FB
:10113000FF0E8CEC18F0FF0E8CEC18F03FB8B7EFF8
:1011400008F048EC30F0FF0E8CEC18F038EC30F082
:10115000FF0E8CEC18F078EC30F0FF0E8CEC18F0F1
:10116000D8EC2FF0FF0E8CEC18F0CBEF08F028EC49
:1011700030F0FF0E8CEC18F098EC2FF0FF0E8CEC9A
:1011800018F0B8EC2FF0FF0E8CEC18F058EC2FF0A4
:10119000FF0E8CEC18F030EC18F05B0E3CEC18F005
:1011A000BA0E64EC18F03FAAEFEF08F0FF0E8CECDB
:1011B00018F0E8EC30F0FF0E8CEC18F078EC2FF023
:1011C000FF0E8CEC18F098EC2FF0FF0E8CEC18F062
:1011D00028EC30F0FF0E8CEC18F006EF09F0000E52
:1011E0008CEC18F008EC31F0000E8CEC18F008ECE8
:1011F00031F0000E8CEC18F008EC31F0000E8CECA5
:1012000018F008EC31F0000E8CEC18F012EC27F01E
:1012100050A0C9EF09F030EC18F0400E3CEC18F08B
:10122000BE0E64EC18F038EC2EF0000E8CEC18F0CA
:10123000000E8CEC18F07CEC31F018EC26F04450E9
:10124000486E4550496E4806000E325CD8A439EF0E
:1012500009F04FB035EF09F0000E485ED8A435EF25
:1012600009F07CEC31F03CEF09F086EC31F03CEF1A
:1012700009F07CEC31F032063A2A120E3A5CD8A41E
:1012800023EF09F03A6A33EC18F0400E3CEC18F00A
:10129000BE0E64EC18F04806000E325CD8A461EF74
:1012A00009F04FB05DEF09F0000E485ED8A45DEF85
:1012B00009F07CEC31F064EF09F086EC31F064EF7A
:1012C00009F07CEC31F032063A2A150E3A5CD8A4CB
:1012D0004BEF09F03A6A12EC27F030EC18F0400EB0
:1012E0003CEC18F0BF0E64EC18F098EC2EF0000EF9
:1012F0008CEC18F0000E8CEC18F07CEC31F0490608
:10130000000E315CD8A495EF09F04FB091EF09F0D1
:10131000000E495ED8A491EF09F07CEC31F098EF13
:1013200009F086EC31F098EF09F07CEC31F03106F1
:101330003A2A120E3A5CD8A47FEF09F03A6A33ECED
:1013400018F0400E3CEC18F0BF0E64EC18F04906A3
:10135000000E315CD8A4BDEF09F04FB0B9EF09F031
:10136000000E495ED8A4B9EF09F07CEC31F0C0EF73
:1013700009F086EC31F0C0EF09F07CEC31F0310679
:101380003A2A150E3A5CD8A4A7EF09F03A6A66EF3C
:1013900001F030EC18F0400E3CEC18F0BE0E64EC9E
:1013A00018F078EC2EF0000E8CEC18F090EC31F088
:1013B00018EC26F04450486E4550496E4806000E21
:1013C000325CD8A4F4EF09F04FB0F0EF09F0000E52
:1013D000485ED8A4F0EF09F090EC31F0F7EF09F097
:1013E00097EC31F0F7EF09F090EC31F032063A2A41
:1013F0001C0E3A5CD8A4DEEF09F03A6A33EC18F020
:10140000400E3CEC18F0BE0E64EC18F078EC2EF0B8
:10141000000E8CEC18F090EC31F04906000E315CB7
:10142000D8A423EF0AF04FB01FEF0AF0000E495E78
:10143000D8A41FEF0AF090EC31F026EF0AF097ECF9
:1014400031F026EF0AF090EC31F031063A2A1C0E0A
:101450003A5CD8A40DEF0AF03A6A30EC18F0400E6E
:101460003CEC18F0BF0E64EC18F058EC2EF0000EB7
:101470008CEC18F090EC31F095EC26F046504A6E6A
:1014800047504B6E4A06000E345CD8A458EF0AF061
:101490004FB054EF0AF0000E4A5ED8A454EF0AF0A1
:1014A00090EC31F05BEF0AF097EC31F05BEF0AF073
:1014B00090EC31F034063A2A1C0E3A5CD8A442EF84
:1014C0000AF03A6A12EC27F033EC18F0400E3CECCC
:1014D00018F0BF0E64EC18F058EC2EF0000E8CECF7
:1014E00018F090EC31F04B06000E335CD8A489EF75
:1014F0000AF04FB085EF0AF0000E4B5ED8A485EFDE
:101500000AF090EC31F08CEF0AF097EC31F08CEFB0
:101510000AF090EC31F033063A2A1C0E3A5CD8A45B
:1015200073EF0AF03A6A66EF01F012EC27F030EC44
:1015300018F0410E3CEC18F0B80E64EC18F0700E88
:101540008CEC18F0100E8CEC18F0100E8CEC18F0DF
:10155000100E8CEC18F0000E8CEC18F078EC2EF0DD
:10156000000E8CEC18F0F8EC2DF0000E8CEC18F05E
:1015700098EC2DF0000E8CEC18F0D8EC2AF0000E50
:101580008CEC18F0E8EC2AF0000E8CEC18F0C8ECAB
:101590002AF0000E8CEC18F0C8EC2AF008EC31F0C0
:1015A000A8EC2EF0000E8CEC18F0D8EC2DF0000E0C
:1015B0008CEC18F033EC18F0400E3CEC18F0B80E40
:1015C00064EC18F0B8EC2EF0000E8CEC18F0B8ECCF
:1015D0002EF0000E8CEC18F018EC2EF0000E8CECB7
:1015E00018F058EC2EF0000E8CEC18F0F8EC2DF002
:1015F000000E8CEC18F0082A210E085CD8B406EF17
:101600000BF0100E8CEC18F0FBEF0AF0086A700E6D
:101610008CEC18F030EC18F0400E3CEC18F0B90EE1
:1016200064EC18F012B01AEF0BF0000E195CD8B48D
:1016300067EF0BF0000E8CEC18F038EC2EF0000E7B
:101640008CEC18F0000E8CEC18F05CEC31F0000E15
:101650008CEC18F0000E8CEC18F098EC2EF008ECE6
:1016600031F0B8EC2DF0000E8CEC18F008EC2EF0F8
:1016700008EC31F0B8EC2DF0000E8CEC18F068ECB2
:101680002EF0000E8CEC18F058EC2EF0000E8CECC6
:1016900018F0B8EC2EF033EC18F0400E3CEC18F0DB
:1016A000B90E64EC18F0000E8CEC18F098EC2EF0EB
:1016B000000E8CEC18F068EC2EF0000E8CEC18F09C
:1016C00038EC2EF0000E8CEC18F0B2EF0BF0FF0EA1
:1016D0008CEC18F008EC30F0FF0E8CEC18F0FF0EDC
:1016E0008CEC18F06CEC31F0FF0E8CEC18F0FF0E67
:1016F0008CEC18F068EC30F018EC31F078EC2FF04E
:10170000FF0E8CEC18F0C8EC2FF018EC31F078ECF0
:101710002FF0FF0E8CEC18F038EC30F0FF0E8CEC54
:1017200018F028EC30F0FF0E8CEC18F088EC30F05C
:1017300033EC18F0400E3CEC18F0B90E64EC18F0E5
:10174000FF0E8CEC18F068EC30F0FF0E8CEC18F00B
:1017500038EC30F0FF0E8CEC18F008EC30F0FF0E97
:101760008CEC18F030EC18F0400E3CEC18F0BB0E8E
:1017700064EC18F012B0C2EF0BF0010E195CD8B493
:1017800005EF0CF0000E8CEC18F018EC2FF0000EAA
:101790008CEC18F0B8EC2DF0000E8CEC18F0D8ECB6
:1017A0002DF0000E8CEC18F058EC2EF008EC31F017
:1017B000A8EC2EF0000E8CEC18F0D8EC2DF0000EFA
:1017C0008CEC18F0B8EC2EF0000E8CEC18F0B8ECA5
:1017D0002EF0000E8CEC18F018EC2EF0000E8CECB5
:1017E00018F058EC2EF033EC18F0400E3CEC18F0EA
:1017F000BB0E64EC18F0000E8CEC18F0F8EC2DF039
:10180000000E8CEC18F046EF0CF0FF0E8CEC18F08C
:10181000E8EC30F0FF0E8CEC18F078EC2FF0FF0EB7
:101820008CEC18F098EC2FF0FF0E8CEC18F028ECF4
:1018300030F018EC31F078EC30F0FF0E8CEC18F052
:1018400098EC2FF0FF0E8CEC18F088EC30F0FF0EC7
:101850008CEC18F088EC30F0FF0E8CEC18F0D8EC23
:101860002FF0FF0E8CEC18F028EC30F033EC18F071
:10187000400E3CEC18F0BB0E64EC18F0FF0E8CEC44
:1018800018F0B8EC2FF0FF0E8CEC18F012EC27F0EB
:1018900030EC18F0430E3CEC18F0BA0E64EC18F083
:1018A0001E0E8CEC18F0100E8CEC18F0100E8CEC58
:1018B00018F0100E8CEC18F0100E8CEC18F030ECC8
:1018C00018F0430E3CEC18F0BC0E64EC18F01E0E41
:1018D0008CEC18F0100E8CEC18F0100E8CEC18F04C
:1018E000100E8CEC18F0100E8CEC18F030EC18F098
:1018F0004A0E3CEC18F0BA0E64EC18F04EB223EF2E
:101900000DF012A089EF0CF0000E195CD8B4D6EFE0
:101910000CF0000E8CEC18F018EC2EF0000E8CEC95
:1019200018F058EC2EF0000E8CEC18F0B8EC2EF0FD
:10193000000E8CEC18F0D8EC2DF0000E8CEC18F0AA
:1019400098EC2EF0000E8CEC18F038EC2EF0000E17
:101950008CEC18F068EC2EF0000E8CEC18F0B8EC63
:101960002DF0000E8CEC18F028EC2EF033EC18F073
:10197000400E3CEC18F0BA0E64EC18F0000E8CEC43
:1019800018F008EC31F008EC31F0000E8CEC18F097
:1019900008EC31F0000E08EC31F0000E08EC31F0EC
:1019A000000E08EC31F0000E4FEF0EF0FF0E8CEC45
:1019B00018F0D8EC2FF0FF0E8CEC18F028EC30F07B
:1019C000FF0E8CEC18F088EC30F0FF0E8CEC18F069
:1019D00098EC2FF0FF0E8CEC18F068EC30F0FF0E56
:1019E0008CEC18F008EC30F0FF0E8CEC18F038ECB2
:1019F00030F0FF0E8CEC18F078EC2FF0FF0E8CEC32
:101A000018F0F8EC2FF033EC18F0400E3CEC18F026
:101A1000BA0E64EC18F0FF0E8CEC18F008EC31F004
:101A200008EC31F0000E8CEC18F008EC31F0000EF0
:101A300008EC31F0000E08EC31F0000E08EC31F04B
:101A4000000E4FEF0EF012A02BEF0DF0000E195C00
:101A5000D8B4BEEF0DF0000E8CEC18F0A8EC2EF010
:101A6000000E8CEC18F0D8EC2DF0000E8CEC18F079
:101A700078EC2EF0000E8CEC18F098EC2DF0000EA7
:101A80008CEC18F098EC2EF0000E8CEC18F098EC22
:101A90002DF0000E8CEC18F0B8EC2EF0000E8CEC53
:101AA00018F0D8EC2DF0000E8CEC18F008EC31F0AA
:101AB00033EC18F0400E3CEC18F0BA0E64EC18F061
:101AC000000E8CEC18F04EA46DEF0DF098EC2EF09B
:101AD000000E8CEC18F072EF0DF038EC2EF0000ECA
:101AE0008CEC18F04EB68DEF0DF008EC31F008ECF0
:101AF00031F0000E8CEC18F008EC31F0000E8CEC9C
:101B000018F008EC31F0000E8CEC18F008EC31F015
:101B1000000E8CEC18F04FEF0EF008EC31F04EB8E0
:101B2000A8EF0DF078EC2EF0000E8CEC18F068ECBD
:101B30002EF0000E8CEC18F0A8EC2EF0000E8CECC1
:101B400018F018EC2EF0000E8CEC18F04FEF0EF0A1
:101B500058EC2EF0000E8CEC18F0D8EC2DF0000EA6
:101B60008CEC18F0F8EC2DF0000E8CEC18F098ECE2
:101B70002DF0000E8CEC18F04FEF0EF0FF0E8CECF9
:101B800018F078EC30F0FF0E8CEC18F098EC2FF099
:101B9000FF0E8CEC18F048EC30F0FF0E8CEC18F0D7
:101BA00058EC2FF0FF0E8CEC18F068EC30F0FF0EC4
:101BB0008CEC18F058EC2FF0FF0E8CEC18F088EC41
:101BC00030F0FF0E8CEC18F098EC2FF0FF0E8CEC40
:101BD00018F018EC31F033EC18F0400E3CEC18F033
:101BE000BA0E64EC18F0FF0E8CEC18F04EA400EF67
:101BF0000EF068EC30F0FF0E8CEC18F005EF0EF0F4
:101C000008EC30F0FF0E8CEC18F04EB620EF0EF022
:101C100008EC31F008EC31F0000E8CEC18F008EC18
:101C200031F0000E8CEC18F008EC31F0000E8CEC6A
:101C300018F008EC31F0000E8CEC18F04FEF0EF0BD
:101C400018EC31F04EB83BEF0EF048EC30F0FF0EE0
:101C50008CEC18F038EC30F0FF0E8CEC18F078ECCF
:101C600030F0FF0E8CEC18F0D8EC2FF0FF0E8CEC5F
:101C700018F04FEF0EF028EC30F0FF0E8CEC18F05F
:101C800098EC2FF0FF0E8CEC18F0B8EC2FF0FF0E54
:101C90008CEC18F058EC2FF0FF0E8CEC18F030ECB8
:101CA00018F04A0E3CEC18F0BC0E64EC18F04EBA7A
:101CB0008AEF0EF012A062EF0EF0010E195CD8B49C
:101CC00076EF0EF0000E8CEC18F068EC2EF0000EA3
:101CD0008CEC18F0E8EC2DF0000E8CEC18F0E8EC31
:101CE0002DF0000E8CEC18F0B8EF0EF0FF0E8CEC1F
:101CF00018F038EC30F0FF0E8CEC18F0A8EC2FF058
:101D0000FF0E8CEC18F0A8EC2FF0FF0E8CEC18F006
:101D1000B8EF0EF012A092EF0EF0010E195CD8B4DD
:101D2000A6EF0EF0000E8CEC18F068EC2EF0000E12
:101D30008CEC18F058EC2EF0000E8CEC18F008EC3F
:101D400031F0000E8CEC18F0B8EF0EF0FF0E8CECBA
:101D500018F038EC30F0FF0E8CEC18F028EC30F076
:101D6000FF0E8CEC18F008EC31F0000E8CEC18F043
:101D700066EF01F012EC27F030EC18F0410E3CEC6D
:101D800018F0B80E64EC18F0700E8CEC18F0100E11
:101D90008CEC18F0100E8CEC18F0100E8CEC18F087
:101DA000000E8CEC18F068EC2EF0000E8CEC18F0A5
:101DB000B8EC2EF0000E8CEC18F008EC2EF0000EB3
:101DC0008CEC18F0D8EC2DF0000E8CEC18F098ECA0
:101DD0002EF008EC31F0A8EC2EF0000E8CEC18F090
:101DE000D8EC2DF0000E8CEC18F0B8EC2EF0000EB4
:101DF0008CEC18F0B8EC2EF033EC18F0400E3CEC04
:101E000018F0B80E64EC18F018EC2EF0000E8CEC04
:101E100018F058EC2EF0000E8CEC18F0F8EC2DF0C9
:101E2000000E8CEC18F0082A2D0E085CD8B41EEFBA
:101E30000FF0100E8CEC18F013EF0FF0086A700E14
:101E40008CEC18F012EC27F030EC18F0400E3CEC63
:101E500018F0B90E64EC18F012B234EF0FF0000E67
:101E60001A5CD8B460EF0FF0000E8CEC18F078EC30
:101E70002EF0000E8CEC18F0D8EC2DF0000E8CEC4F
:101E800018F098EC2DF0000E8CEC18F028EC2EF0E9
:101E900008EC31F008EC2EF0000E8CEC18F068EC39
:101EA0002EF0000E8CEC18F038EC2EF0000E8CECBE
:101EB00018F0C8EC2DF0000E8CEC18F08AEF0FF043
:101EC000FF0E8CEC18F048EC30F0FF0E8CEC18F0A4
:101ED00098EC2FF0FF0E8CEC18F058EC2FF0FF0E62
:101EE0008CEC18F0F8EC2FF018EC31F0C8EC2FF077
:101EF000FF0E8CEC18F038EC30F0FF0E8CEC18F084
:101F000008EC30F0FF0E8CEC18F088EC2FF0FF0E90
:101F10008CEC18F030EC18F0430E3CEC18F0BA0ED4
:101F200064EC18F01E0E8CEC18F0100E8CEC18F00F
:101F3000100E8CEC18F0100E8CEC18F0100E8CECCF
:101F400018F030EC18F0400E3CEC18F0BD0E64ECCC
:101F500018F012B2B1EF0FF0020E1A5CD8B409EF0C
:101F600010F0000E8CEC18F038EC2EF0000E8CEC1B
:101F700018F0D8EC2DF0000E8CEC18F0D8EC2EF008
:101F8000000E8CEC18F0D8EC2DF0000E8CEC18F054
:101F900038EC2EF008EC31F048EC2EF0000E8CEC12
:101FA00018F0B8EC2EF008EC31F098EC2EF0000EA2
:101FB0008CEC18F0B8EC2EF0000E8CEC18F0000E43
:101FC0008CEC18F033EC18F0400E3CEC18F0BD0E21
:101FD00064EC18F0000E8CEC18F0000E8CEC18F08D
:101FE000000E8CEC18F0B8EC2EF0000E8CEC18F013
:101FF00018EC2EF0000E8CEC18F048EC2EF0000ED1
:102000008CEC18F0D8EC2DF0000E8CEC18F05FEF93
:1020100010F0FF0E8CEC18F008EC30F0FF0E8CEC9A
:1020200018F098EC2FF0FF0E8CEC18F0A8EC30F0C4
:10203000FF0E8CEC18F098EC2FF0FF0E8CEC18F0E3
:1020400008EC30F018EC31F018EC30F0FF0E8CECAE
:1020500018F088EC30F018EC31F068EC30F0FF0E3E
:102060008CEC18F088EC30F0FF0E8CEC18F0FF0EC2
:102070008CEC18F033EC18F0400E3CEC18F0BD0E70
:1020800064EC18F0FF0E8CEC18F0FF0E8CEC18F0DE
:10209000FF0E8CEC18F088EC30F0FF0E8CEC18F092
:1020A000D8EC2FF0FF0E8CEC18F018EC30F0FF0E8F
:1020B0008CEC18F098EC2FF0FF0E8CEC18F030EC54
:1020C00018F0430E3CEC18F0BE0E64EC18F01E0E37
:1020D0008CEC18F0100E8CEC18F0100E8CEC18F044
:1020E000100E8CEC18F0100E8CEC18F012EC27F09F
:1020F00030EC18F0400E3CEC18F0BB0E64EC18F01D
:1021000012B288EF10F0010E1A5CD8B4B9EF10F0DB
:10211000000E8CEC18F078EC2EF0000E8CEC18F021
:10212000D8EC2DF0000E8CEC18F098EC2DF0000E91
:102130008CEC18F028EC2EF008EC31F098EC2EF036
:10214000000E8CEC18F0D8EC2DF0000E8CEC18F092
:10215000A8EC2EF0000E8CEC18F0D8EC2DF0000E50
:102160008CEC18F0B8EC2EF0000E8CEC18F0E8EFC8
:1021700010F0FF0E8CEC18F048EC30F0FF0E8CECF9
:1021800018F098EC2FF0FF0E8CEC18F058EC2FF0B4
:10219000FF0E8CEC18F0F8EC2FF018EC31F068EC36
:1021A00030F0FF0E8CEC18F098EC2FF0FF0E8CEC5A
:1021B00018F078EC30F0FF0E8CEC18F098EC2FF063
:1021C000FF0E8CEC18F088EC30F0FF0E8CEC18F061
:1021D00012EC27F030EC18F0430E3CEC18F0BC0E7B
:1021E00064EC18F01E0E8CEC18F0100E8CEC18F04D
:1021F000100E8CEC18F0100E8CEC18F0100E8CEC0D
:1022000018F030EC18F04A0E3CEC18F0BA0E64EC02
:1022100018F051B046EF11F0000E1A5CD8A414EF7C
:1022200011F012B22DEF11F0000E8CEC18F008EC4A
:102230002EF0000E8CEC18F068EC2EF0000E8CECFA
:1022400018F038EC2EF0000E8CEC18F0C8EC2DF0E5
:10225000000E8CEC18F07EEF11F0FF0E8CEC18F0F5
:10226000C8EC2FF0FF0E8CEC18F038EC30F0FF0EBD
:102270008CEC18F008EC30F0FF0E8CEC18F088ECC9
:102280002FF0FF0E8CEC18F07EEF11F0000E1A5CB0
:10229000D8A44EEF11F012B267EF11F0000E8CECE3
:1022A00018F0E8EC2DF0000E8CEC18F098EC2EF005
:1022B000000E8CEC18F0D8EC2DF0000E8CEC18F021
:1022C000D8EC2DF0000E8CEC18F07EEF11F0FF0E24
:1022D0008CEC18F0A8EC2FF0FF0E8CEC18F068ECEA
:1022E00030F0FF0E8CEC18F098EC2FF0FF0E8CEC19
:1022F00018F098EC2FF0FF0E8CEC18F030EC18F082
:102300004A0E3CEC18F0BE0E64EC18F0000E5B5C5C
:10231000D8B4DEEF11F0010E5B5CD8B42CEF12F0F4
:10232000020E1A5CD8A498EF11F012B2BBEF11F0B4
:10233000000E8CEC18F0A8EC2EF0000E8CEC18F0CF
:1023400038EC2EF0000E8CEC18F068EC2EF0000E3D
:102350008CEC18F0E8EC2EF0000E8CEC18F008EC89
:1023600031F0000E8CEC18F008EC31F0000E8CEC23
:1023700018F078EF12F0FF0E8CEC18F078EC30F0DB
:10238000FF0E8CEC18F008EC30F0FF0E8CEC18F01F
:1023900038EC30F0FF0E8CEC18F0B8EC30F0FF0E9B
:1023A0008CEC18F008EC31F0000E8CEC18F008EC16
:1023B00031F0000E8CEC18F078EF12F0020E1A5C7F
:1023C000D8A4E6EF11F012B209EF12F0000E8CEC77
:1023D00018F0E8EC2DF0000E8CEC18F098EC2DF0D5
:1023E000000E8CEC18F0A8EC2EF0000E8CEC18F01F
:1023F000B8EC2EF0000E8CEC18F008EC31F0000E6A
:102400008CEC18F008EC31F0000E8CEC18F078EF42
:1024100012F0FF0E8CEC18F0A8EC2FF0FF0E8CECF5
:1024200018F058EC2FF0FF0E8CEC18F078EC30F030
:10243000FF0E8CEC18F088EC30F0FF0E8CEC18F0EE
:1024400008EC31F0000E8CEC18F008EC31F0000EC6
:102450008CEC18F078EF12F0020E1A5CD8A434EF6E
:1024600012F012B257EF12F0000E8CEC18F058EC8C
:102470002EF0000E8CEC18F068EC2EF0000E8CECB8
:1024800018F098EC2EF0000E8CEC18F048EC2EF0C2
:10249000000E8CEC18F098EC2DF0000E8CEC18F07F
:1024A00038EC2EF0000E8CEC18F078EF12F0FF0EE6
:1024B0008CEC18F028EC30F0FF0E8CEC18F038ECB7
:1024C00030F0FF0E8CEC18F068EC30F0FF0E8CEC66
:1024D00018F018EC30F0FF0E8CEC18F058EC2FF0E0
:1024E000FF0E8CEC18F008EC30F0FF0E8CEC18F0BE
:1024F00012EC27F030EC18F04A0E3CEC18F0BC0E51
:1025000064EC18F051B2E7EF12F0010E1A5CD8A497
:102510008DEF12F012B2BAEF12F0000E8CEC18F040
:10252000B8EC2EF0000E8CEC18F018EC2EF0000E2B
:102530008CEC18F048EC2EF0000E8CEC18F0D8EC77
:102540002DF008EC31F068EC2EF0000E8CEC18F059
:10255000C8EC2EF0000E8CEC18F0B8EC2EF0000E4B
:102560008CEC18F0000E8CEC18F0000E8CEC18F0CF
:1025700047EF13F0FF0E8CEC18F088EC30F0FF0EF4
:102580008CEC18F0D8EC2FF0FF0E8CEC18F018EC57
:1025900030F0FF0E8CEC18F098EC2FF018EC31F0C6
:1025A00038EC30F0FF0E8CEC18F098EC30F0FF0EA9
:1025B0008CEC18F088EC30F0FF0E8CEC18F0000E6C
:1025C0008CEC18F0000E8CEC18F047EF13F0010EB5
:1025D0001A5CD8A4EFEF12F012B21CEF13F0000E49
:1025E0008CEC18F0C8EC2DF0000E8CEC18F0D8EC48
:1025F0002DF0000E8CEC18F0B8EC2DF0000E8CECE9
:1026000018F098EC2EF0000E8CEC18F0D8EC2DF0B1
:10261000000E8CEC18F098EC2DF0000E8CEC18F0FD
:10262000A8EC2EF0000E8CEC18F0D8EC2DF0000E7B
:102630008CEC18F047EF13F0FF0E8CEC18F088ECE0
:102640002FF0FF0E8CEC18F098EC2FF0FF0E8CECB6
:1026500018F078EC2FF0FF0E8CEC18F068EC30F0EE
:10266000FF0E8CEC18F098EC2FF0FF0E8CEC18F0AD
:1026700058EC2FF0FF0E8CEC18F078EC30F0FF0ED9
:102680008CEC18F098EC2FF0FF0E8CEC18F012EC9C
:1026900027F030EC18F0460E3CEC18F0BF0E64EC5E
:1026A00018F0A8EC2EF0000E8CEC18F068EC2EF070
:1026B000000E8CEC18F0E8EC2DF0000E8CEC18F00D
:1026C000B8EC2EF0000E8CEC18F0E8EC2EF0000EBA
:1026D0008CEC18F098EC2DF0000E8CEC18F098ECC7
:1026E0002EF0000E8CEC18F0D8EC2DF0000E8CECD7
:1026F00018F008EC31F0D8EC2EF033EC18F0400E66
:102700003CEC18F0BF0E64EC18F0000E8CEC18F0E6
:10271000D8EC2DF0000E8CEC18F098EC2EF0000E9A
:102720008CEC18F0A8EC2EF0000E8CEC18F018ECE5
:102730002EF0000E8CEC18F068EC2EF0000E8CECF5
:1027400018F058EC2EF0000E8CEC18F008EC31F07C
:10275000000E8CEC18F0C8EC2AF0000E8CEC18F08F
:10276000000E8CEC18F0400E8CEC18F0000E8CEC87
:1027700018F0B8EC2AF0000E8CEC18F0B8EC2AF047
:10278000000E8CEC18F066EF01F012EC27F030EC44
:1027900018F0410E3CEC18F0B80E64EC18F0700E16
:1027A0008CEC18F0100E8CEC18F0100E8CEC18F06D
:1027B000100E8CEC18F0000E8CEC18F0D8EC2DF00C
:1027C000000E8CEC18F0D8EC2DF0000E8CEC18F00C
:1027D00078EC2EF0000E8CEC18F098EC2EF0000E39
:1027E0008CEC18F068EC2EF0000E8CEC18F048EC35
:1027F0002EF008EC31F0E8EC2EF0000E8CEC18F026
:1028000098EC2EF0000E8CEC18F018EC2EF033EC57
:1028100018F0400E3CEC18F0B80E64EC18F0B8EC70
:102820002EF0000E8CEC18F0D8EC2DF0000E8CEC95
:1028300018F0082A330E085CD8B424EF14F0100EF8
:102840008CEC18F019EF14F0086A700E8CEC18F08C
:1028500012EC27F030EC18F0400E3CEC18F0B90EFA
:1028600064EC18F012B43AEF14F0000E1B5CD8B40C
:102870007DEF14F0000E8CEC18F0D8EC2DF0000E6B
:102880008CEC18F0D8EC2DF0000E8CEC18F078ECF5
:102890002EF0000E8CEC18F098EC2EF0000E8CEC64
:1028A00018F068EC2EF0000E8CEC18F048EC2EF0CE
:1028B00008EC31F0E8EC2EF0000E8CEC18F098ECFF
:1028C0002EF0000E8CEC18F018EC2EF0000E8CECB4
:1028D00018F0B8EC2EF033EC18F0400E3CEC18F089
:1028E000B90E64EC18F0000E8CEC18F0D8EC2DF05A
:1028F000000E8CEC18F0BEEF14F0FF0E8CEC18F00C
:1029000098EC2FF0FF0E8CEC18F098EC2FF0FF0EE7
:102910008CEC18F048EC30F0FF0E8CEC18F068EC02
:1029200030F0FF0E8CEC18F038EC30F0FF0E8CEC31
:1029300018F018EC30F018EC31F0B8EC30F0FF0E75
:102940008CEC18F068EC30F0FF0E8CEC18F0D8EC42
:102950002FF0FF0E8CEC18F088EC30F033EC18F010
:10296000400E3CEC18F0B90E64EC18F0FF0E8CEC45
:1029700018F098EC2FF0FF0E8CEC18F030EC18F0FB
:10298000430E3CEC18F0BA0E64EC18F01E0E8CEC02
:1029900018F0100E8CEC18F0100E8CEC18F0100ED5
:1029A0008CEC18F0100E8CEC18F030EC18F0400E97
:1029B0003CEC18F0BD0E64EC18F012B4E5EF14F026
:1029C000020E1B5CD8B428EF15F0000E8CEC18F04A
:1029D000C8EC2DF0000E8CEC18F0D8EC2DF0000EA9
:1029E0008CEC18F0E8EC2DF0000E8CEC18F098EC64
:1029F0002DF0000E8CEC18F0C8EC2EF0000E8CECD4
:102A000018F038EC2EF0000E8CEC18F0B8EC2EF02C
:102A100008EC31F038EC2EF0000E8CEC18F068EC7D
:102A20002EF0000E8CEC18F098EC2DF033EC18F032
:102A3000400E3CEC18F0BD0E64EC18F0000E8CEC6F
:102A400018F0C8EC2DF0000E8CEC18F069EF15F0C2
:102A5000FF0E8CEC18F088EC2FF0FF0E8CEC18F0C9
:102A600098EC2FF0FF0E8CEC18F0A8EC2FF0FF0E76
:102A70008CEC18F058EC2FF0FF0E8CEC18F098EC62
:102A800030F0FF0E8CEC18F008EC30F0FF0E8CEC00
:102A900018F088EC30F018EC31F008EC30F0FF0E54
:102AA0008CEC18F038EC30F0FF0E8CEC18F058EC91
:102AB0002FF033EC18F0400E3CEC18F0BD0E64EC37
:102AC00018F0FF0E8CEC18F088EC2FF0FF0E8CEC59
:102AD00018F030EC18F0430E3CEC18F0BE0E64EC2D
:102AE00018F01E0E8CEC18F0100E8CEC18F0100E76
:102AF0008CEC18F0100E8CEC18F0100E8CEC18F01A
:102B000030EC18F0400E3CEC18F0BB0E64EC18F002
:102B100012B490EF15F0010E1B5CD8B4FAEF15F06B
:102B2000000E8CEC18F0D8EC2EF0000E8CEC18F0A7
:102B300068EC2EF0000E8CEC18F038EC2EF008EC5F
:102B400031F0D8EC2EF0000E8CEC18F098EC2DF053
:102B5000000E8CEC18F038EC2EF0000E8CEC18F017
:102B6000C8EC2EF0000E8CEC18F0D8EC2DF008EC30
:102B700031F0A8EC2EF0000E8CEC18F0780E8CECF6
:102B800018F033EC18F0400E3CEC18F0BB0E64EC7F
:102B900018F0140E8CEC18F0120E8CEC18F0140EC9
:102BA0008CEC18F0780E8CEC18F0000E8CEC18F011
:102BB000D8EC2EF0000E8CEC18F0D8EC2DF0000EB6
:102BC0008CEC18F008EC31F0E8EC2DF0000E8CECF9
:102BD00018F038EC2EF0000E8CEC18F098EC2DF07C
:102BE000000E8CEC18F0F8EC2DF0000E8CEC18F0C8
:102BF00062EF16F0FF0E8CEC18F0A8EC30F0FF0E30
:102C00008CEC18F038EC30F0FF0E8CEC18F008EC7F
:102C100030F018EC31F0A8EC30F0FF0E8CEC18F02E
:102C200058EC2FF0FF0E8CEC18F008EC30F0FF0E93
:102C30008CEC18F098EC30F0FF0E8CEC18F098EC5F
:102C40002FF018EC31F078EC30F0FF0E8CEC18F02F
:102C5000870E8CEC18F033EC18F0400E3CEC18F0BA
:102C6000BB0E64EC18F0EB0E8CEC18F0ED0E8CEC57
:102C700018F0EB0E8CEC18F0870E8CEC18F0FF0EB1
:102C80008CEC18F0A8EC30F0FF0E8CEC18F098ECFF
:102C90002FF0FF0E8CEC18F018EC31F0A8EC2FF0B0
:102CA000FF0E8CEC18F008EC30F0FF0E8CEC18F0F6
:102CB00058EC2FF0FF0E8CEC18F0B8EC2FF0FF0E54
:102CC0008CEC18F030EC18F0430E3CEC18F0BC0E15
:102CD00064EC18F01E0E8CEC18F0100E8CEC18F052
:102CE000100E8CEC18F0100E8CEC18F0100E8CEC12
:102CF00018F030EC18F04A0E3CEC18F0BA0E64EC08
:102D000018F053B0D2EF16F0000E1B5CD8A48CEF75
:102D100016F012B4AFEF16F0000E8CEC18F0B8EC11
:102D20002DF0000E8CEC18F098EC2DF0000E8CECD1
:102D300018F058EC2EF0000E8CEC18F0B8EC2DF0DA
:102D4000000E8CEC18F0D8EC2DF0000E8CEC18F086
:102D500038EC2EF0000E8CEC18F01EEF17F0FF0E82
:102D60008CEC18F078EC2FF0FF0E8CEC18F058EC8F
:102D70002FF0FF0E8CEC18F028EC30F0FF0E8CECEE
:102D800018F078EC2FF0FF0E8CEC18F098EC2FF088
:102D9000FF0E8CEC18F008EC30F0FF0E8CEC18F005
:102DA0001EEF17F0000E1B5CD8A4DAEF16F012B479
:102DB000FDEF16F0000E8CEC18F0E8EC2EF0000E93
:102DC0008CEC18F098EC2EF0000E8CEC18F018EC4F
:102DD0002EF0000E8CEC18F0B8EC2EF0000E8CECFF
:102DE00018F0D8EC2DF0000E8CEC18F008EC31F057
:102DF000000E8CEC18F01EEF17F0FF0E8CEC18F0A4
:102E0000B8EC30F0FF0E8CEC18F068EC30F0FF0EF0
:102E10008CEC18F0D8EC2FF0FF0E8CEC18F088EC4E
:102E200030F0FF0E8CEC18F098EC2FF0FF0E8CECCD
:102E300018F008EC31F0000E8CEC18F012EC27F0D2
:102E400030EC18F04A0E3CEC18F0BE0E64EC18F0B2
:102E500053B279EF17F0020E1B5CD8A433EF17F0D2
:102E600012B456EF17F0000E8CEC18F0B8EC2DF001
:102E7000000E8CEC18F098EC2DF0000E8CEC18F095
:102E800058EC2EF0000E8CEC18F0B8EC2DF0000E83
:102E90008CEC18F0D8EC2DF0000E8CEC18F038EC1F
:102EA0002EF0000E8CEC18F0C5EF17F0FF0E8CEC36
:102EB00018F078EC2FF0FF0E8CEC18F058EC2FF097
:102EC000FF0E8CEC18F028EC30F0FF0E8CEC18F0B4
:102ED00078EC2FF0FF0E8CEC18F098EC2FF0FF0E32
:102EE0008CEC18F008EC30F0FF0E8CEC18F0C5EF0D
:102EF00017F0020E1B5CD8A481EF17F012B4A4EFF8
:102F000017F0000E8CEC18F038EC2EF0000E8CEC64
:102F100018F068EC2EF0000E8CEC18F098EC2DF008
:102F2000000E8CEC18F0C8EC2DF0000E8CEC18F0B4
:102F300008EC31F0000E8CEC18F008EC31F0000ECB
:102F40008CEC18F0C5EF17F0FF0E8CEC18F008ECC5
:102F500030F0FF0E8CEC18F038EC30F0FF0E8CECFB
:102F600018F058EC2FF0FF0E8CEC18F088EC2FF0D6
:102F7000FF0E8CEC18F008EC31F0000E8CEC18F021
:102F800008EC31F0000E8CEC18F030EC18F04A0E22
:102F90003CEC18F0BC0E64EC18F04EBC00EF18F0DE
:102FA000010E1B5CD8A4D8EF17F012B4ECEF17F0A9
:102FB000000E8CEC18F068EC2EF0000E8CEC18F083
:102FC000E8EC2DF0000E8CEC18F0E8EC2DF0000E83
:102FD0008CEC18F02EEF18F0FF0E8CEC18F038EC9B
:102FE00030F0FF0E8CEC18F0A8EC2FF0FF0E8CECFC
:102FF00018F0A8EC2FF0FF0E8CEC18F02EEF18F064
:10300000010E1B5CD8A408EF18F012B41CEF18F0E6
:10301000000E8CEC18F068EC2EF0000E8CEC18F022
:1030200058EC2EF0000E8CEC18F008EC31F0000E8D
:103030008CEC18F02EEF18F0FF0E8CEC18F038EC3A
:1030400030F0FF0E8CEC18F028EC30F0FF0E8CEC1A
:1030500018F008EC31F0000E8CEC18F066EF01F07F
:103060008C888C9A12008C988C8A12008C888C8A9E
:1030700012008C988C9A1200016EB7EC18F0015077
:103080008B6E8C928C90000000000000000000000D
:10309000000000000000000000008C840000000020
:1030A0000000000000000000000000000000000020
:1030B0008C940000000000000000000000000000F0
:1030C0000000000000001200026EB7EC18F0025081
:1030D0008B6E8C928C9000000000000000000000BD
:1030E000000000000000000000008C8400000000D0
:1030F00000000000000000000000000000000000D0
:103100008C9400000000000000000000000000009F
:103110000000000000001200006EB7EC18F012BEB4
:10312000F5EC18F000508B6E8C928C800000000043
:10313000000000000000000000000000000000008F
:103140008C8400000000000000000000000000006F
:103150000000000000008C9400000000000000004F
:1031600000000000000000000000000012000F013D
:10317000FF0E946E00018C828C9000000000000015
:1031800000000000000000000000000000008C842F
:10319000000000000000000000000000000000002F
:1031A000000000000000000000000000000000001F
:1031B00000000000000000008C94000000000000EF
:1031C00000000000000000000000000000000000FF
:1031D000000000000000000081BEC7EF18F08C92D4
:1031E0000F01000E946E00011200000E1F5CD8B497
:1031F0001AEF19F0010E1F5CD8B433EF19F0020E6C
:103200001F5CD8B44AEF19F0030E1F5CD8B45FEF0F
:1032100019F0040E1F5CD8B472EF19F0050E1F5C94
:10322000D8B483EF19F0060E1F5CD8B492EF19F0F2
:103230009FEF19F01EB028EF19F000420042004243
:103240000042004200420042010E00169FEF19F0BA
:103250000046004600460046004600460046800EF6
:1032600000169FEF19F01EB040EF19F00042004227
:103270000042004200420042030E00169FEF19F088
:10328000004600460046004600460046C00E0016B6
:103290009FEF19F01EB056EF19F0004200420042B5
:1032A00000420042070E00169FEF19F0004600464C
:1032B000004600460046E00E00169FEF19F01EB0D3
:1032C0006AEF19F000420042004200420F0E001661
:1032D0009FEF19F00046004600460046F00E00162B
:1032E0009FEF19F01EB07CEF19F00042004200423F
:1032F0001F0E00169FEF19F0004600460046F80E1C
:1033000000169FEF19F01EB08CEF19F0004200423A
:103310003F0E00169FEF19F000460046FC0E001607
:103320009FEF19F01EB09AEF19F000427F0E0016C1
:103330009FEF19F00046FE0E00169FEF19F01200E5
:1033400036EC18F0400E3CEC18F0B80E64EC18F0B7
:10335000000E8CEC18F0012A800E015CD8A4A8EFB6
:1033600019F0022A65EC18F0400E3CEC18F0C00E83
:10337000025CD8A4A8EF19F01200106E000E105CC9
:10338000D8A4DBEF19F005B8CCEF19F005BAD0EFEF
:1033900019F018EC2AF0120008EC31F0058C12003C
:1033A00005BCD7EF19F0059C18EC2AF01200059C1B
:1033B00008EC31F01200010E105CD8A4E3EF19F014
:1033C00028EC2AF01200020E105CD8A4EBEF19F0E2
:1033D00038EC2AF01200030E105CD8A4F3EF19F0B9
:1033E00048EC2AF01200040E105CD8A4FBEF19F090
:1033F00058EC2AF01200050E105CD8A403EF1AF066
:1034000068EC2AF01200060E105CD8A40BEF1AF03C
:1034100078EC2AF01200070E105CD8A413EF1AF013
:1034200088EC2AF01200080E105CD8A41BEF1AF0EA
:1034300098EC2AF01200A8EC2AF01200106E000E90
:10344000105CD8A427EF1AF0B8EC2AF01200010E95
:10345000105CD8A42FEF1AF0C8EC2AF01200020E6C
:10346000105CD8A437EF1AF0D8EC2AF01200030E43
:10347000105CD8A43FEF1AF0E8EC2AF01200040E1A
:10348000105CD8A447EF1AF0F8EC2AF01200050EF1
:10349000105CD8A44FEF1AF008EC2BF01200060EC7
:1034A000105CD8A457EF1AF018EC2BF01200070E9E
:1034B000105CD8A45FEF1AF028EC2BF01200080E75
:1034C000105CD8A467EF1AF038EC2BF0120048EC2F
:1034D0002BF01200106E000E105CD8A473EF1AF0DF
:1034E00058EC2BF01200010E105CD8A47BEF1AF000
:1034F00068EC2BF01200020E105CD8A483EF1AF0D7
:1035000078EC2BF01200030E105CD8A48BEF1AF0AD
:1035100088EC2BF01200040E105CD8A493EF1AF084
:1035200098EC2BF01200050E105CD8A49BEF1AF05B
:10353000A8EC2BF01200060E105CD8A4A3EF1AF032
:10354000B8EC2BF01200070E105CD8A4ABEF1AF009
:10355000C8EC2BF01200080E105CD8A4B3EF1AF0E0
:10356000D8EC2BF01200E8EC2BF01200062A0A0E21
:10357000065CD8A4B6EF1AF0066A1200062AFF0EFF
:10358000065CD8A4BEEF1AF0066A072A550E075C3F
:10359000D8A4BEEF1AF0066A076A1200062AFF0EC8
:1035A000065CD8A4CEEF1AF0066A072AFF0E075C65
:1035B000D8A4CEEF1AF0066A076A120030EC18F0B1
:1035C000400E3CEC18F0BF0E64EC18F0D8EC2EF076
:1035D000000E8CEC18F068EC2EF0000E8CEC18F05D
:1035E00038EC2EF0000E8CEC18F0D8EC2AF0000E1F
:1035F0008CEC18F0E8EC2AF0000E8CEC18F0C8EC1B
:103600002AF0000E8CEC18F0C8EC2AF0000E8CECBE
:1036100018F0C8EC2DF008EC31F098EC2EF0000E0C
:103620008CEC18F0D8EC2DF033EC18F0400E3CEC9C
:1036300018F0BF0E64EC18F0D8EC2EF0000E8CECF5
:1036400018F0400E8CEC18F0000E8CEC18F0C8EC62
:103650002AF0000E8CEC18F0400E8CEC18F0000EE6
:103660008CEC18F0B8EC2AF0000E8CEC18F0400E40
:10367000036E7F0E046E30EC18F003503CEC18F033
:10368000BC0E64EC18F0010E8CEC18F033EC18F062
:1036900004503CEC18F0BC0E64EC18F0010E8CECFD
:1036A00018F0032A0406BEEC1AF0BEEC1AF0800EE5
:1036B000035CD8A43BEF1BF0CEEC1AF0CEEC1AF072
:1036C000CEEC1AF0CEEC1AF0CEEC1AF0CEEC1AF0EA
:1036D000CEEC1AF0CEEC1AF0CEEC1AF0BEEC1AF0EA
:1036E000400E036E7F0E046E30EC18F003503CEC7D
:1036F00018F0BC0E64EC18F0000E8CEC18F033ECF3
:1037000018F004503CEC18F0BC0E64EC18F0000EFD
:103710008CEC18F0032A0406BEEC1AF0BEEC1AF08A
:10372000800E035CD8A474EF1BF0128ECEEC1AF05E
:10373000CEEC1AF0CEEC1AF0CEEC1AF0CEEC1AF079
:10374000CEEC1AF0CEEC1AF0BEEC1AF01E8030EC83
:1037500018F04A0E3CEC18F0BB0E64EC18F048EC84
:103760002CF0000E8CEC18F0100E8CEC18F0100EF3
:103770008CEC18F0100E8CEC18F0100E8CEC18F08D
:10378000100E8CEC18F0000E8CEC18F0C8EC2CF03D
:10379000000E8CEC18F008EC31F0000E8CEC18F0F8
:1037A00038EC2CF0000E8CEC18F0C8EC2CF0000E6D
:1037B0008CEC18F058EC2CF0000E8CEC18F078EC37
:1037C0002CF0000E8CEC18F0C8EC2CF0000E8CECF9
:1037D00018F033EC18F0400E3CEC18F0BB0E64EC23
:1037E00018F038EC2CF0000E8CEC18F038EC2CF0C3
:1037F000000E8CEC18F008EC2DF0000E8CEC18F09C
:1038000078EC2CF0000E8CEC18F0C8EC2CF0000ECC
:103810008CEC18F058EC2CF0000E8CEC18F01E908C
:1038200030EC18F0560E3CEC18F0BC0E64EC18F0BE
:10383000F8EC2BF0000E8CEC18F038EC2DF0000EAC
:103840008CEC18F028EC2CF0000E8CEC18F078ECD6
:103850002CF0000E8CEC18F0D8EC2CF0000E8CEC58
:1038600018F008EC31F0000E8CEC18F0A8EC2CF0FD
:10387000000E8CEC18F033EC18F0400E3CEC18F015
:10388000BC0E64EC18F0F8EC2BF0000E8CEC18F089
:1038900008EC2CF0000E8CEC18F0D8EC2CF0000E9C
:1038A0008CEC18F008EC2DF0000E8CEC18F0F8EC15
:1038B0002BF0000E8CEC18F028EC2DF0000E8CECA8
:1038C00018F0D8EC2CF0000E8CEC18F008EC2DF071
:1038D000000E8CEC18F078EC2DF0000E8CEC18F04B
:1038E0001F2A080E1F5CD8A496EF1BF0129E1F6AB9
:1038F000CEEC1AF0CEEC1AF0CEEC1AF0CEEC1AF0B8
:10390000CEEC1AF0CEEC1AF0CEEC1AF0CEEC1AF0A7
:10391000CEEC1AF0CEEC1AF0CEEC1AF0CEEC1AF097
:10392000CEEC1AF0CEEC1AF0CEEC1AF0CEEC1AF087
:10393000CEEC1AF0CEEC1AF0CEEC1AF0CEEC1AF077
:10394000CEEC1AF0CEEC1AF0CEEC1AF0CEEC1AF067
:10395000CEEC1AF0CEEC1AF0CEEC1AF0CEEC1AF057
:10396000CEEC1AF0CEEC1AF0CEEC1AF0CEEC1AF047
:10397000CEEC1AF0CEEC1AF0CEEC1AF0CEEC1AF037
:10398000CEEC1AF0CEEC1AF0CEEC1AF0CEEC1AF027
:10399000CEEC1AF0CEEC1AF0CEEC1AF0CEEC1AF017
:1039A000CEEC1AF0CEEC1AF0CEEC1AF0CEEC1AF007
:1039B000CEEC1AF0CEEC1AF0CEEC1AF0CEEC1AF0F7
:1039C000CEEC1AF0CEEC1AF0CEEC1AF0CEEC1AF0E7
:1039D000CEEC1AF0CEEC1AF0CEEC1AF0CEEC1AF0D7
:1039E000CEEC1AF0CEEC1AF0CEEC1AF0CEEC1AF0C7
:1039F000CEEC1AF0CEEC1AF0CEEC1AF0CEEC1AF0B7
:103A0000CEEC1AF0CEEC1AF0CEEC1AF0CEEC1AF0A6
:103A1000CEEC1AF0CEEC1AF0CEEC1AF0CEEC1AF096
:103A2000CEEC1AF0CEEC1AF0CEEC1AF0CEEC1AF086
:103A3000CEEC1AF0CEEC1AF0CEEC1AF0CEEC1AF076
:103A4000CEEC1AF0CEEC1AF0CEEC1AF0CEEC1AF066
:103A5000CEEC1AF0CEEC1AF0CEEC1AF0CEEC1AF056
:103A6000CEEC1AF0CEEC1AF0CEEC1AF0CEEC1AF046
:103A7000CEEC1AF0CEEC1AF0CEEC1AF0CEEC1AF036
:103A8000CEEC1AF0CEEC1AF0CEEC1AF0CEEC1AF026
:103A9000CEEC1AF0CEEC1AF0A0EC19F0CEEC1AF045
:103AA000CEEC1AF0CEEC1AF0CEEC1AF0CEEC1AF006
:103AB000CEEC1AF0CEEC1AF0CEEC1AF0CEEC1AF0F6
:103AC000CEEC1AF01200096E640E095ED8A06CEFFD
:103AD0001DF00A2A64EF1DF0640E09260A0E095E25
:103AE000D8A076EF1DF00B2A6EEF1DF00A0E092606
:103AF000010E095ED8A080EF1DF00C2A78EF1DF0B2
:103B000012000D6E100E0D5ED8A08AEF1DF00B2A6C
:103B100082EF1DF0100E0D26010E0D5ED8A094EF61
:103B20001DF00C2A8CEF1DF0120005880A50BDEC28
:103B300019F0000E8CEC18F00598058A0B50BDECBE
:103B400019F0000E8CEC18F0059A0C50BDEC19F031
:103B5000000E8CEC18F00A6A0B6A0C6A12000A500C
:103B60001EEC1AF0000E8CEC18F00B501EEC1AF044
:103B7000000E8CEC18F00C501EEC1AF0000E8CECC1
:103B800018F00A6A0B6A0C6A12000A506AEC1AF002
:103B9000FF0E8CEC18F00B506AEC1AF0FF0E8CEC58
:103BA00018F00C506AEC1AF0FF0E8CEC18F00A6A50
:103BB0000B6A0C6A1200136E182A090E185CD8B42E
:103BC000F1EF1DF013BEE9EF1DF0B8EC2AF0EBEFBA
:103BD0001DF0C8EC2AF0000E8CEC18F01346DCEF58
:103BE0001DF0186A1200136E080E185CD8B430EF7E
:103BF0001EF013BE15EF1EF018501C5CD8B40BEF6E
:103C00001EF0000E8CEC18F0B8EC2AF0000E8CECD4
:103C100018F02CEF1EF0FF0E8CEC18F058EC2BF087
:103C2000FF0E8CEC18F02CEF1EF018501C5CD8B472
:103C300024EF1EF0000E8CEC18F0C8EC2AF0000EF9
:103C40008CEC18F02CEF1EF0FF0E8CEC18F068ECEA
:103C50002BF0FF0E8CEC18F0182A1346F4EF1DF031
:103C6000186A1200010EC26EC28AC286C284C28263
:103C7000C2B238EF1EF0000EC26EC4502A6EC3509E
:103C8000296E010EC26EC284C282C2B245EF1EF01E
:103C9000C4502C6EC3502B6E000EC26E12EC27F077
:103CA000010EC26EC28AC288C284C282C2B256EFFC
:103CB0001EF0C4502E6EC3502D6E000EC26E010E4B
:103CC000C26EC294C282C2B263EF1EF0C450306EA4
:103CD000C3502F6E000EC26E50B073EC1EF050A099
:103CE00055EC21F012002AB27AEF1EF02A1E030EC4
:103CF0002A16291E2AB0AAEF1FF0030E295CD8B09D
:103D000086EF1EF0000E326EE2EF1FF0050E295C0A
:103D1000D8B08FEF1EF0010E326EE2EF1FF0070EEB
:103D2000295CD8B098EF1EF0020E326EE2EF1FF061
:103D3000080E295CD8B0A1EF1EF0030E326EE2EF40
:103D40001FF0090E295CD8B0AAEF1EF0040E326EE7
:103D5000E2EF1FF00A0E295CD8B0B3EF1EF0050E9B
:103D6000326EE2EF1FF00B0E295CD8B0BCEF1EF0F4
:103D7000060E326EE2EF1FF00D0E295CD8B0C5EFD3
:103D80001EF0070E326EE2EF1FF00E0E295CD8B067
:103D9000CEEF1EF0080E326EE2EF1FF0100E295C1F
:103DA000D8B0D7EF1EF0090E326EE2EF1FF0120E00
:103DB000295CD8B0E0EF1EF00A0E326EE2EF1FF081
:103DC000140E295CD8B0E9EF1EF00B0E326EE2EF54
:103DD0001FF0170E295CD8B0F2EF1EF00C0E326EF9
:103DE000E2EF1FF0190E295CD8B0FBEF1EF00D0EAC
:103DF000326EE2EF1FF01D0E295CD8B004EF1FF009
:103E00000E0E326EE2EF1FF0200E295CD8B00DEFDF
:103E10001FF00F0E326EE2EF1FF0240E295CD8B0B7
:103E200016EF1FF0100E326EE2EF1FF0290E295C24
:103E3000D8B01FEF1FF0110E326EE2EF1FF02E0E02
:103E4000295CD8B028EF1FF0120E326EE2EF1FF09F
:103E5000330E295CD8B031EF1FF0130E326EE2EF53
:103E60001FF0390E295CD8B03AEF1FF0140E326EF5
:103E7000E2EF1FF0400E295CD8B043EF1FF0150EA3
:103E8000326EE2EF1FF0490E295CD8B04CEF1FF004
:103E9000160E326EE2EF1FF0510E295CD8B055EFCE
:103EA0001FF0170E326EE2EF1FF05B0E295CD8B0E8
:103EB0005EEF1FF0180E326EE2EF1FF0660E295C07
:103EC000D8B067EF1FF0190E326EE2EF1FF0720EDE
:103ED000295CD8B070EF1FF01A0E326EE2EF1FF0BF
:103EE000800E295CD8B079EF1FF01B0E326EE2EF26
:103EF0001FF0900E295CD8B082EF1FF01C0E326EBE
:103F0000E2EF1FF0A10E295CD8B08BEF1FF01D0E61
:103F1000326EE2EF1FF0B50E295CD8B094EF1FF0BF
:103F20001E0E326EE2EF1FF0CB0E295CD8B09DEF73
:103F30001FF01F0E326EE2EF1FF0E40E295CD8B0C6
:103F4000A6EF1FF0200E326EE2EF1FF0210E326E50
:103F5000E2EF1FF0000E295CD8A4B3EF1FF0210E92
:103F6000326EE2EF1FF01F0E295CD8B0BCEF1FF0DD
:103F7000220E326EE2EF1FF0420E295CD8B0C5EF80
:103F80001FF0230E326EE2EF1FF06A0E295CD8B0EC
:103F9000CEEF1FF0240E326EE2EF1FF0960E295C7A
:103FA000D8B0D7EF1FF0250E326EE2EF1FF0C70E2C
:103FB000295CD8B0E0EF1FF0260E326EE2EF1FF062
:103FC000270E326E2CB2E9EF1FF02C1E030E2C16BA
:103FD0002B1E2CB019EF21F0030E2B5CD8B0F5EF9F
:103FE0001FF0000E316E53EF21F0050E2B5CD8B0A0
:103FF000FEEF1FF0010E316E53EF21F0070E2B5C28
:10400000D8B007EF20F0020E316E53EF21F0080E0A
:104010002B5CD8B010EF20F0030E316E53EF21F07F
:10402000090E2B5CD8B019EF20F0040E316E53EF5F
:1040300021F00A0E2B5CD8B022EF20F0050E316E75
:1040400053EF21F00B0E2B5CD8B02BEF20F0060EB7
:10405000316E53EF21F00D0E2B5CD8B034EF20F011
:10406000070E316E53EF21F00E0E2B5CD8B03DEFF2
:1040700020F0080E316E53EF21F0100E2B5CD8B0FB
:1040800046EF20F0090E316E53EF21F0120E2B5C3B
:10409000D8B04FEF20F00A0E316E53EF21F0140E1E
:1040A0002B5CD8B058EF20F00B0E316E53EF21F09F
:1040B000170E2B5CD8B061EF20F00C0E316E53EF71
:1040C00021F0190E2B5CD8B06AEF20F00D0E316E86
:1040D00053EF21F01D0E2B5CD8B073EF20F00E0EC5
:1040E000316E53EF21F0200E2B5CD8B07CEF20F026
:1040F0000F0E316E53EF21F0240E2B5CD8B085EFFC
:1041000020F0100E316E53EF21F0290E2B5CD8B049
:104110008EEF20F0110E316E53EF21F02E0E2B5C3E
:10412000D8B097EF20F0120E316E53EF21F0330E1E
:104130002B5CD8B0A0EF20F0130E316E53EF21F0BE
:10414000390E2B5CD8B0A9EF20F0140E316E53EF6E
:1041500021F0400E2B5CD8B0B2EF20F0150E316E7E
:1041600053EF21F0490E2B5CD8B0BBEF20F0160EB8
:10417000316E53EF21F0510E2B5CD8B0C4EF20F01C
:10418000170E316E53EF21F05B0E2B5CD8B0CDEFE4
:1041900020F0180E316E53EF21F0660E2B5CD8B074
:1041A000D6EF20F0190E316E53EF21F0720E2B5C1A
:1041B000D8B0DFEF20F01A0E316E53EF21F0800EF1
:1041C0002B5CD8B0E8EF20F01B0E316E53EF21F0DE
:1041D000900E2B5CD8B0F1EF20F01C0E316E53EF37
:1041E00021F0A10E2B5CD8B0FAEF20F01D0E316E3D
:1041F00053EF21F0B50E2B5CD8B003EF21F01E0E6B
:10420000316E53EF21F0CB0E2B5CD8B00CEF21F0C8
:104210001F0E316E53EF21F0E40E2B5CD8B015EF7A
:1042200021F0200E316E53EF21F0210E316E53EF4D
:1042300021F0000E2B5CD8A422EF21F0210E316E6C
:1042400053EF21F01F0E2B5CD8B02BEF21F0220E84
:10425000316E53EF21F0420E2B5CD8B034EF21F0D9
:10426000230E316E53EF21F06A0E2B5CD8B03DEF78
:1042700021F0240E316E53EF21F0960E2B5CD8B056
:1042800046EF21F0250E316E53EF21F0C70E2B5C67
:10429000D8B04FEF21F0260E316E53EF21F0270EEC
:1042A000316E53EF21F066EF25F02AB25CEF21F07A
:1042B0002A1E030E2A16291E2AB020EF22F0030E12
:1042C000295CD8B068EF21F0000E326E58EF22F072
:1042D000050E295CD8B071EF21F0010E326E58EF57
:1042E00022F0070E295CD8B07AEF21F0020E326E70
:1042F00058EF22F0080E295CD8B083EF21F0030EAE
:10430000326E58EF22F00A0E295CD8B08CEF21F003
:10431000040E326E58EF22F00D0E295CD8B095EFE6
:1043200021F0050E326E58EF22F0100E295CD8B045
:104330009EEF21F0060E326E58EF22F0140E295C2B
:10434000D8B0A7EF21F0070E326E58EF22F0190E09
:10435000295CD8B0B0EF21F0080E326E58EF22F091
:10436000200E295CD8B0B9EF21F0090E326E58EF5B
:1043700022F0290E295CD8B0C2EF21F00A0E326E6D
:1043800058EF22F0330E295CD8B0CBEF21F00B0EA2
:10439000326E58EF22F0400E295CD8B0D4EF21F0F5
:1043A0000C0E326E58EF22F0510E295CD8B0DDEFC2
:1043B00021F00D0E326E58EF22F0660E295CD8B057
:1043C000E6EF21F00E0E326E58EF22F0800E295CDF
:1043D000D8B0EFEF21F00F0E326E58EF22F0900EB2
:1043E000295CD8B0F8EF21F0100E326E58EF22F0B1
:1043F000A10E295CD8B001EF22F0110E326E58EFF9
:1044000022F0B50E295CD8B00AEF22F0120E326EFF
:1044100058EF22F0CB0E295CD8B013EF22F0130E28
:10442000326E58EF22F0E40E295CD8B01CEF22F077
:10443000140E326E58EF22F0150E326E58EF22F045
:10444000000E295CD8A429EF22F0150E326E58EF29
:1044500022F01F0E295CD8B032EF22F0160E326E19
:1044600058EF22F0420E295CD8B03BEF22F0170E35
:10447000326E58EF22F06A0E295CD8B044EF22F079
:10448000180E326E58EF22F0960E295CD8B04DEF20
:1044900022F0190E326E58EF22F0C70E295CD8B008
:1044A00056EF22F01A0E326E58EF22F01B0E326ECB
:1044B0002CB25FEF22F02C1E030E2C162B1E2CB0FC
:1044C00023EF23F0030E2B5CD8B06BEF22F0000E2D
:1044D000316E5BEF23F0050E2B5CD8B074EF22F049
:1044E000010E316E5BEF23F0070E2B5CD8B07DEF31
:1044F00022F0020E316E5BEF23F0080E2B5CD8B079
:1045000086EF22F0030E316E5BEF23F00A0E2B5C78
:10451000D8B08FEF22F0040E316E5BEF23F00D0E5A
:104520002B5CD8B098EF22F0050E316E5BEF23F0D4
:10453000100E2B5CD8B0A1EF22F0060E316E5BEFAF
:1045400023F0140E2B5CD8B0AAEF22F0070E316EC8
:104550005BEF23F0190E2B5CD8B0B3EF22F0080EFE
:10456000316E5BEF23F0200E2B5CD8B0BCEF22F055
:10457000090E316E5BEF23F0290E2B5CD8B0C5EF2E
:1045800022F00A0E316E5BEF23F0330E2B5CD8B0B5
:10459000CEEF22F00B0E316E5BEF23F0400E2B5C62
:1045A000D8B0D7EF22F00C0E316E5BEF23F0510E36
:1045B0002B5CD8B0E0EF22F00D0E316E5BEF23F0F4
:1045C000660E2B5CD8B0E9EF22F00E0E316E5BEF79
:1045D00023F0800E2B5CD8B0F2EF22F00F0E316E7C
:1045E0005BEF23F0900E2B5CD8B0FBEF22F0100EA7
:1045F000316E5BEF23F0A10E2B5CD8B004EF23F0FB
:10460000110E316E5BEF23F0B50E2B5CD8B00DEFC1
:1046100023F0120E316E5BEF23F0CB0E2B5CD8B083
:1046200016EF23F0130E316E5BEF23F0E40E2B5CDC
:10463000D8B01FEF23F0140E316E5BEF23F0150E90
:10464000316E5BEF23F0000E2B5CD8A42CEF23F02F
:10465000150E316E5BEF23F01F0E2B5CD8B035EFDB
:1046600023F0160E316E5BEF23F0420E2B5CD8B0B8
:104670003EEF23F0170E316E5BEF23F06A0E2B5CDA
:10468000D8B047EF23F0180E316E5BEF23F0960E93
:104690002B5CD8B050EF23F0190E316E5BEF23F096
:1046A000C70E2B5CD8B059EF23F01A0E316E5BEFBA
:1046B00023F01B0E316E2EB262EF23F02E1E030E7E
:1046C0002E162D1E2EB026EF24F0030E2D5CD8B032
:1046D0006EEF23F0000E346E5EEF24F0050E2D5CBD
:1046E000D8B077EF23F0010E346E5EEF24F0070EA2
:1046F0002D5CD8B080EF23F0020E346E5EEF24F014
:10470000080E2D5CD8B089EF23F0030E346E5EEFF7
:1047100024F00A0E2D5CD8B092EF23F0040E346E14
:104720005EEF24F00D0E2D5CD8B09BEF23F0050E4C
:10473000346E5EEF24F0100E2D5CD8B0A4EF23F0A1
:10474000060E346E5EEF24F0140E2D5CD8B0ADEF83
:1047500023F0070E346E5EEF24F0190E2D5CD8B0F6
:10476000B6EF23F0080E346E5EEF24F0200E2D5CC1
:10477000D8B0BFEF23F0090E346E5EEF24F0290E9F
:104780002D5CD8B0C8EF23F00A0E346E5EEF24F033
:10479000330E2D5CD8B0D1EF23F00B0E346E5EEFEC
:1047A00024F0400E2D5CD8B0DAEF23F00C0E346EFE
:1047B0005EEF24F0510E2D5CD8B0E3EF23F00D0E28
:1047C000346E5EEF24F0660E2D5CD8B0ECEF23F073
:1047D0000E0E346E5EEF24F0800E2D5CD8B0F5EF37
:1047E00023F00F0E346E5EEF24F0900E2D5CD8B0E7
:1047F000FEEF23F0100E346E5EEF24F0A10E2D5C60
:10480000D8B007EF24F0110E346E5EEF24F0B50E31
:104810002D5CD8B010EF24F0120E346E5EEF24F051
:10482000CB0E2D5CD8B019EF24F0130E346E5EEF72
:1048300024F0E40E2D5CD8B022EF24F0140E346E78
:104840005EEF24F0150E346E5EEF24F0000E2D5C4A
:10485000D8A42FEF24F0150E346E5EEF24F01F0E57
:104860002D5CD8B038EF24F0160E346E5EEF24F0D5
:10487000420E2D5CD8B041EF24F0170E346E5EEF7F
:1048800024F06A0E2D5CD8B04AEF24F0180E346E76
:104890005EEF24F0960E2D5CD8B053EF24F0190E85
:1048A000346E5EEF24F0C70E2D5CD8B05CEF24F0C0
:1048B0001A0E346E5EEF24F01B0E346E30B265EFCC
:1048C00024F0301E030E30162F1E30B029EF25F0D5
:1048D000030E2F5CD8B071EF24F0000E336E61EF41
:1048E00025F0050E2F5CD8B07AEF24F0010E336E60
:1048F00061EF25F0070E2F5CD8B083EF24F0020E95
:10490000336E61EF25F0080E2F5CD8B08CEF24F0E9
:10491000030E336E61EF25F00A0E2F5CD8B095EFD1
:1049200024F0040E336E61EF25F00D0E2F5CD8B02D
:104930009EEF24F0050E336E61EF25F0100E2F5C14
:10494000D8B0A7EF24F0060E336E61EF25F0140EF9
:104950002F5CD8B0B0EF24F0070E336E61EF25F076
:10496000190E2F5CD8B0B9EF24F0080E336E61EF4A
:1049700025F0200E2F5CD8B0C2EF24F0090E336E64
:1049800061EF25F0290E2F5CD8B0CBEF24F00A0E92
:10499000336E61EF25F0330E2F5CD8B0D4EF24F0E6
:1049A0000B0E336E61EF25F0400E2F5CD8B0DDEFBB
:1049B00024F00C0E336E61EF25F0510E2F5CD8B051
:1049C000E6EF24F00D0E336E61EF25F0660E2F5CDE
:1049D000D8B0EFEF24F00E0E336E61EF25F0800EAD
:1049E0002F5CD8B0F8EF24F00F0E336E61EF25F096
:1049F000900E2F5CD8B001EF25F0100E336E61EFF2
:104A000025F0A10E2F5CD8B00AEF25F0110E336E01
:104A100061EF25F0B50E2F5CD8B013EF25F0120E24
:104A2000336E61EF25F0CB0E2F5CD8B01CEF25F074
:104A3000130E336E61EF25F0E40E2F5CD8B025EF36
:104A400025F0140E336E61EF25F0150E336E61EF15
:104A500025F0000E2F5CD8A432EF25F0150E336E32
:104A600061EF25F01F0E2F5CD8B03BEF25F0160E3E
:104A7000336E61EF25F0420E2F5CD8B044EF25F085
:104A8000170E336E61EF25F06A0E2F5CD8B04DEF34
:104A900025F0180E336E61EF25F0960E2F5CD8B01E
:104AA00056EF25F0190E336E61EF25F0C70E2F5C1F
:104AB000D8B05FEF25F01A0E336E61EF25F01B0EB4
:104AC000336E66EC25F0BFEC25F012003650325CF8
:104AD000D8B08FEF25F0000E365CD8B48FEF25F0FC
:104AE0003C2A000E5A5CD8A479EF25F0010E82EF23
:104AF00025F0010E5A5CD8A481EF25F0020E82EF5A
:104B000025F0030E3C5CD8A48BEF25F0360636501A
:104B1000326E8FEF25F03650326E90EF25F03C6A02
:104B20003550315CD8B0BAEF25F0000E355CD8B402
:104B3000BAEF25F03B2A000E5A5CD8A4A3EF25F06B
:104B4000010EACEF25F0010E5A5CD8A4ABEF25F0B6
:104B5000020EACEF25F0030E3B5CD8A4B5EF25F0B8
:104B600035063550316EB9EF25F03550316EBAEF5C
:104B700025F03B6A3250366E3150356E1200385097
:104B8000345CD8B0E8EF25F0000E385CD8B4E8EF1C
:104B900025F03E2A000E5A5CD8A4D2EF25F0010E73
:104BA000DBEF25F0010E5A5CD8A4DAEF25F0020EF7
:104BB000DBEF25F0030E3E5CD8A4E4EF25F03806C9
:104BC0003850346EE8EF25F03850346EE9EF25F0B8
:104BD0003E6A3750335CD8B013EF26F0000E375CD6
:104BE000D8B413EF26F03D2A000E5A5CD8A4FCEF8F
:104BF00025F0010E05EF26F0010E5A5CD8A404EF53
:104C000026F0020E05EF26F0030E3D5CD8A40EEF51
:104C100026F037063750336E12EF26F03750336EDA
:104C200013EF26F03D6A3450386E3350376E120061
:104C30004FB246EF26F04550315CD8A025EF26F064
:104C40003150456E416A30EF26F06E0E415CD8B4AB
:104C50002DEF26F0412A30EF26F0416A3150456EA3
:104C60004450325CD8A03AEF26F03250446E406A8D
:104C700045EF26F06E0E405CD8B442EF26F0402A95
:104C800045EF26F0406A3250446E12004550315CC8
:104C9000D8A051EF26F03150456E416A1E926DEF5B
:104CA00026F01EB25CEF26F0460E415CD8B45CEFF5
:104CB00026F0412A6DEF26F0416A1E82000E455C07
:104CC000D8B46DEF26F0080E5D5CD8B46BEF26F01B
:104CD0005D2A6DEF26F05D6A45064450325CD8A02F
:104CE00078EF26F03250446E406A1E9494EF26F01E
:104CF0001EB483EF26F0460E405CD8B483EF26F056
:104D0000402A94EF26F0406A1E84000E445CD8B41A
:104D100094EF26F0080E5C5CD8B492EF26F05C2A83
:104D200094EF26F05C6A440612004FB2C3EF26F0FF
:104D30004750335CD8A0A2EF26F03350476E436A49
:104D4000ADEF26F06E0E435CD8B4AAEF26F0432AEE
:104D5000ADEF26F0436A3350476E4650345CD8A01E
:104D6000B7EF26F03450466E426AC2EF26F06E0E60
:104D7000425CD8B4BFEF26F0422AC2EF26F0426A66
:104D80003450466E12004750335CD8A0CEEF26F068
:104D90003350476E436A1E96EAEF26F01EB6D9EFEF
:104DA00026F0460E435CD8B4D9EF26F0432AEAEF4A
:104DB00026F0436A1E86000E475CD8B4EAEF26F060
:104DC000080E5F5CD8B4E8EF26F05F2AEAEF26F021
:104DD0005F6A47064650345CD8A0F5EF26F03450A1
:104DE000466E426A1E9811EF27F01EB800EF27F0BA
:104DF000460E425CD8B400EF27F0422A11EF27F0AC
:104E0000426A1E88000E465CD8B411EF27F0080EE7
:104E10005E5CD8B40FEF27F05E2A11EF27F05E6AD0
:104E20004606120080A818EF27F0228019EF27F01D
:104E3000229080AA1FEF27F0228220EF27F02292F3
:104E4000030E225CD8B4118C000E225CD8A4BBEFF8
:104E500028F011ACBBEF28F0119C020E235CD8A403
:104E6000F4EF27F0000E145CD8B443EF27F0010EE6
:104E7000145CD8B447EF27F0020E145CD8B4A4EF4A
:104E800027F0CDEF27F054EC29F0BBEF28F012B05B
:104E900052EF27F0000E195CD8B4BBEF28F01906CA
:104EA000BBEF28F0000E195CD8B459EF27F0A0EF43
:104EB00027F04E501E0B136E1E0E135CD8B47CEF01
:104EC00027F00E0E135CD8B482EF27F01A0E135C95
:104ED000D8B488EF27F00A0E135CD8B48EEF27F011
:104EE000060E135CD8B494EF27F0020E135CD8B40E
:104EF0009AEF27F0BBEF28F04E824E844E864E98F4
:104F0000BBEF28F04E824E944E864E88BBEF28F0C1
:104F10004E824E944E864E98BBEF28F04E824E84C1
:104F20004E964E98BBEF28F04E824E944E964E9879
:104F3000BBEF28F04E924E944E964E98BBEF28F061
:104F40004EBA4E9ABBEF28F012B2AFEF27F0000E28
:104F50001A5CD8B4BBEF28F01A06BBEF28F0000E9D
:104F60001A5CD8A4BAEF27F051B0BBEF28F05180FB
:104F7000BBEF28F0010E1A5CD8B4C7EF27F0020E81
:104F80005B5CD8B4BBEF28F05B2ABBEF28F051A2E2
:104F9000BBEF28F05192BBEF28F012B4D8EF27F006
:104FA000000E1B5CD8B4BBEF28F01B06BBEF28F04B
:104FB000000E1B5CD8A4E3EF27F053A0BBEF28F052
:104FC0005390BBEF28F0020E1B5CD8A4EEEF27F045
:104FD00053A2BBEF28F05392BBEF28F04EACBBEFCF
:104FE00028F04E9CBBEF28F0010E235CD8A4BBEF49
:104FF00028F0000E145CD8B40AEF28F0010E145CFF
:10500000D8B40EEF28F0020E145CD8B46BEF28F081
:1050100094EF28F0C2EC28F0BBEF28F012B019EFA3
:1050200028F0010E195CD8B4BBEF28F0192ABBEFA9
:1050300028F0000E195CD8B420EF28F067EF28F0B4
:105040004E501E0B136E000E135CD8B443EF28F0C5
:10505000020E135CD8B449EF28F0060E135CD8B4E6
:105060004FEF28F00A0E135CD8B455EF28F01A0E53
:10507000135CD8B45BEF28F00E0E135CD8B461EF6C
:1050800028F0BBEF28F04E824E944E964E98BBEF20
:1050900028F04E824E844E964E98BBEF28F04E82FA
:1050A0004E944E864E98BBEF28F04E824E944E861C
:1050B0004E88BBEF28F04E824E844E864E98BBEF52
:1050C00028F04E824E844E864E88BBEF28F04EAAC2
:1050D0004E8ABBEF28F012B276EF28F0020E1A5C6F
:1050E000D8B4BBEF28F01A2ABBEF28F0000E1A5CE8
:1050F000D8A481EF28F051A0BBEF28F05190BBEF6E
:1051000028F0010E1A5CD8B48EEF28F0000E5B5C1C
:10511000D8B4BBEF28F05B06BBEF28F051B2BBEF71
:1051200028F05182BBEF28F012B49FEF28F0020E56
:105130001B5CD8B4BBEF28F01B2ABBEF28F0000E95
:105140001B5CD8A4AAEF28F053B0BBEF28F0538023
:10515000BBEF28F0020E1B5CD8A4B5EF28F053B2C9
:10516000BBEF28F05382BBEF28F04EBCBBEF28F01A
:105170004E8CBBEF28F02250236EFF0E4C5CD8A45F
:105180004C2A12002D0E4C5CD8B0CBEF28F0080E44
:105190004D6EF1EF28F0410E4C5CD8B0D4EF28F002
:1051A000050E4D6EF1EF28F0550E4C5CD8B0DDEFDA
:1051B00028F0030E4D6EF1EF28F0690E4C5CD8B06C
:1051C000E6EF28F0060E4D6EF1EF28F07D0E4C5CF8
:1051D000D8B0EFEF28F0030E4D6EF1EF28F0010E7E
:1051E0004D6E4D50526E3FA2FCEF28F03FB423EFBE
:1051F00029F03FB811EF29F0FF0E245CD8A404EF8A
:1052000029F04C6A0CEF29F0242A5206000E525C59
:10521000D8A4FCEF28F04C6A4D50526E3FB623EFF5
:1052200029F0FF0E255CD8A419EF29F04C6A21EF74
:1052300029F0252A5206000E525CD8A411EF29F05D
:105240004C6A4D50526E3FA22CEF29F03FA451EF13
:1052500029F03FB841EF29F0FF0E265CD8A434EFC7
:1052600029F04C6A3CEF29F0262A5206000E525CC7
:10527000D8A42CEF29F04C6A4D50526E3FB651EF36
:1052800029F0FF0E275CD8A449EF29F04C6A51EFB2
:1052900029F0272A5206000E525CD8A441EF29F0CB
:1052A0004C6AE6EC29F012002D0E4C5CD8B05DEF94
:1052B00029F0080E4D6E83EF29F0410E4C5CD8B0FA
:1052C00066EF29F0050E4D6E83EF29F0550E4C5C0C
:1052D000D8B06FEF29F0030E4D6E83EF29F0690E01
:1052E0004C5CD8B078EF29F0060E4D6E83EF29F0B4
:1052F0007D0E4C5CD8B081EF29F0030E4D6E83EF2C
:1053000029F0010E4D6E4D50526E3FA28EEF29F0E6
:105310003FB4B5EF29F03FB8A3EF29F0000E245CAD
:10532000D8A496EF29F04C6A9EEF29F02406520685
:10533000000E525CD8A48EEF29F04C6A4D50526E8C
:105340003FB6B5EF29F0000E255CD8A4ABEF29F0ED
:105350004C6AB3EF29F025065206000E525CD8A421
:10536000A3EF29F04C6A4D50526E3FA2BEEF29F0D8
:105370003FA4E3EF29F03FB8D3EF29F0000E265CFD
:10538000D8A4C6EF29F04C6ACEEF29F026065206C3
:10539000000E525CD8A4BEEF29F04C6A4D50526EFC
:1053A0003FB6E3EF29F0000E275CD8A4DBEF29F02D
:1053B0004C6AE3EF29F027065206000E525CD8A48F
:1053C000D3EF29F04C6AE6EC29F012008A922450BF
:1053D000F5EC29F02550F5EC29F02650F5EC29F0F4
:1053E0002750F5EC29F08A821200206E00000000A0
:1053F0000000000000008A9620AE02EF2AF08A84A6
:1054000006EF2AF08A940000000000008A8600005F
:1054100000000000000000008A9600000000204606
:10542000212A080E215CD8A4FCEF29F0216A120081
:105430007C0E8CEC18F0820E8CEC18F0820E8CEC4A
:1054400018F0820E8CEC18F07C0E8CEC18F0120028
:10545000000E8CEC18F0840E8CEC18F0FE0E8CEC28
:1054600018F0800E8CEC18F0000E8CEC18F0120086
:10547000E20E8CEC18F0920E8CEC18F0920E8CEC84
:1054800018F0920E8CEC18F08C0E8CEC18F01200C8
:10549000440E8CEC18F0820E8CEC18F0920E8CEC12
:1054A00018F0920E8CEC18F06C0E8CEC18F01200C8
:1054B000300E8CEC18F0280E8CEC18F0240E8CECCE
:1054C00018F0FE0E8CEC18F0200E8CEC18F0120088
:1054D0004E0E8CEC18F08A0E8CEC18F08A0E8CECC8
:1054E00018F08A0E8CEC18F0720E8CEC18F012008A
:1054F0007C0E8CEC18F0920E8CEC18F0920E8CEC6A
:1055000018F0920E8CEC18F0640E8CEC18F012006F
:10551000060E8CEC18F0020E8CEC18F0C20E8CEC1F
:1055200018F0320E8CEC18F00E0E8CEC18F0120005
:105530006C0E8CEC18F0920E8CEC18F0920E8CEC39
:1055400018F0920E8CEC18F06C0E8CEC18F0120027
:105550004C0E8CEC18F0920E8CEC18F0920E8CEC39
:1055600018F0920E8CEC18F07C0E8CEC18F01200F7
:105570003C0E8CEC18F0420E8CEC18F0420E8CECC9
:1055800018F0420E8CEC18F03C0E8CEC18F0120067
:10559000000E8CEC18F0440E8CEC18F07E0E8CECA7
:1055A00018F0400E8CEC18F0000E8CEC18F0120085
:1055B000720E8CEC18F04A0E8CEC18F04A0E8CEC43
:1055C00018F04A0E8CEC18F0440E8CEC18F0120017
:1055D000220E8CEC18F04A0E8CEC18F04A0E8CEC73
:1055E00018F04A0E8CEC18F0340E8CEC18F0120007
:1055F000300E8CEC18F0280E8CEC18F0240E8CEC8D
:1056000018F07E0E8CEC18F0200E8CEC18F01200C6
:105610002E0E8CEC18F04A0E8CEC18F04A0E8CEC26
:1056200018F04A0E8CEC18F0320E8CEC18F01200C8
:105630003C0E8CEC18F04A0E8CEC18F04A0E8CECF8
:1056400018F04A0E8CEC18F0300E8CEC18F01200AA
:10565000060E8CEC18F0020E8CEC18F0620E8CEC3E
:1056600018F0120E8CEC18F00E0E8CEC18F01200E4
:10567000340E8CEC18F04A0E8CEC18F04A0E8CECC0
:1056800018F04A0E8CEC18F0340E8CEC18F0120066
:105690000C0E8CEC18F0520E8CEC18F0520E8CECB8
:1056A00018F0520E8CEC18F03C0E8CEC18F0120036
:1056B000C30E8CEC18F0BD0E8CEC18F0BD0E8CEC0B
:1056C00018F0BD0E8CEC18F0C30E8CEC18F0120024
:1056D000FF0E8CEC18F0BB0E8CEC18F0810E8CECED
:1056E00018F0BF0E8CEC18F0FF0E8CEC18F01200C6
:1056F0008D0E8CEC18F0B50E8CEC18F0B50E8CEC11
:1057000018F0B50E8CEC18F0BB0E8CEC18F01200F3
:10571000DD0E8CEC18F0B50E8CEC18F0B50E8CECA0
:1057200018F0B50E8CEC18F0CB0E8CEC18F01200C3
:10573000CF0E8CEC18F0D70E8CEC18F0DB0E8CEC46
:1057400018F0810E8CEC18F0DF0E8CEC18F01200C3
:10575000D10E8CEC18F0B50E8CEC18F0B50E8CEC6C
:1057600018F0B50E8CEC18F0CD0E8CEC18F0120081
:10577000C30E8CEC18F0B50E8CEC18F0B50E8CEC5A
:1057800018F0B50E8CEC18F0CF0E8CEC18F012005F
:10579000F90E8CEC18F0FD0E8CEC18F09D0E8CECD4
:1057A00018F0ED0E8CEC18F0F10E8CEC18F01200E5
:1057B000CB0E8CEC18F0B50E8CEC18F0B50E8CEC12
:1057C00018F0B50E8CEC18F0CB0E8CEC18F0120023
:1057D000F30E8CEC18F0AD0E8CEC18F0AD0E8CECDA
:1057E00018F0AD0E8CEC18F0C30E8CEC18F0120013
:1057F000F80E8CEC18F0240E8CEC18F0220E8CECC9
:1058000018F0240E8CEC18F0F80E8CEC18F0120046
:10581000FE0E8CEC18F0920E8CEC18F0920E8CECC4
:1058200018F0920E8CEC18F06C0E8CEC18F0120044
:105830007C0E8CEC18F0820E8CEC18F0820E8CEC46
:1058400018F0820E8CEC18F0440E8CEC18F012005C
:10585000FE0E8CEC18F0820E8CEC18F0820E8CECA4
:1058600018F0820E8CEC18F07C0E8CEC18F0120004
:10587000FE0E8CEC18F0920E8CEC18F0920E8CEC64
:1058800018F0920E8CEC18F0820E8CEC18F01200CE
:10589000FE0E8CEC18F0120E8CEC18F0120E8CEC44
:1058A00018F0120E8CEC18F0020E8CEC18F01200AE
:1058B0007C0E8CEC18F0820E8CEC18F0820E8CECC6
:1058C00018F0920E8CEC18F0740E8CEC18F012009C
:1058D000FE0E8CEC18F0100E8CEC18F0100E8CEC08
:1058E00018F0100E8CEC18F0FE0E8CEC18F0120074
:1058F000000E8CEC18F0820E8CEC18F0FE0E8CEC86
:1059000018F0820E8CEC18F0000E8CEC18F01200DF
:10591000600E8CEC18F0800E8CEC18F0800E8CEC85
:1059200018F0800E8CEC18F07E0E8CEC18F0120043
:10593000FE0E8CEC18F0100E8CEC18F0280E8CEC8F
:1059400018F0440E8CEC18F0820E8CEC18F012005B
:10595000FE0E8CEC18F0800E8CEC18F0800E8CECA7
:1059600018F0800E8CEC18F0800E8CEC18F0120001
:10597000FE0E8CEC18F0040E8CEC18F0080E8CEC7B
:1059800018F0040E8CEC18F0FE0E8CEC18F01200DF
:10599000FE0E8CEC18F0080E8CEC18F0100E8CEC4F
:1059A00018F0200E8CEC18F0FE0E8CEC18F01200A3
:1059B0007C0E8CEC18F0820E8CEC18F0820E8CECC5
:1059C00018F0820E8CEC18F07C0E8CEC18F01200A3
:1059D000FE0E8CEC18F0120E8CEC18F0120E8CEC03
:1059E00018F0120E8CEC18F00C0E8CEC18F0120063
:1059F0007C0E8CEC18F0820E8CEC18F0A20E8CEC65
:105A000018F0420E8CEC18F0BC0E8CEC18F0120062
:105A1000FE0E8CEC18F0120E8CEC18F0120E8CECC2
:105A200018F0120E8CEC18F0EC0E8CEC18F0120042
:105A30004C0E8CEC18F0920E8CEC18F0920E8CEC54
:105A400018F0920E8CEC18F0640E8CEC18F012002A
:105A5000020E8CEC18F0020E8CEC18F0FE0E8CECA2
:105A600018F0020E8CEC18F0020E8CEC18F01200FC
:105A70007E0E8CEC18F0800E8CEC18F0800E8CEC06
:105A800018F0800E8CEC18F07E0E8CEC18F01200E2
:105A90000E0E8CEC18F0300E8CEC18F0C00E8CEC66
:105AA00018F0300E8CEC18F00E0E8CEC18F0120082
:105AB0001E0E8CEC18F0E00E8CEC18F0180E8CEC2E
:105AC00018F0E00E8CEC18F01E0E8CEC18F01200A2
:105AD000C60E8CEC18F0280E8CEC18F0100E8CEC26
:105AE00018F0280E8CEC18F0C60E8CEC18F0120092
:105AF0000E0E8CEC18F0100E8CEC18F0E00E8CEC06
:105B000018F0100E8CEC18F00E0E8CEC18F0120041
:105B1000C20E8CEC18F0A20E8CEC18F0920E8CECED
:105B200018F08A0E8CEC18F0860E8CEC18F012002F
:105B3000780E8CEC18F0140E8CEC18F0120E8CEC25
:105B400018F0140E8CEC18F0780E8CEC18F0120093
:105B50007E0E8CEC18F04A0E8CEC18F04A0E8CEC91
:105B600018F04A0E8CEC18F0340E8CEC18F0120081
:105B70003C0E8CEC18F0420E8CEC18F0420E8CECC3
:105B800018F0420E8CEC18F0240E8CEC18F0120079
:105B90007E0E8CEC18F0420E8CEC18F0420E8CEC61
:105BA00018F0420E8CEC18F03C0E8CEC18F0120041
:105BB0007E0E8CEC18F04A0E8CEC18F04A0E8CEC31
:105BC00018F04A0E8CEC18F0420E8CEC18F0120013
:105BD0007E0E8CEC18F00A0E8CEC18F00A0E8CEC91
:105BE00018F00A0E8CEC18F0020E8CEC18F0120073
:105BF0003C0E8CEC18F0420E8CEC18F0420E8CEC43
:105C000018F0520E8CEC18F0340E8CEC18F01200D8
:105C10007E0E8CEC18F0080E8CEC18F0080E8CEC54
:105C200018F0080E8CEC18F07E0E8CEC18F01200B8
:105C3000000E8CEC18F0420E8CEC18F07E0E8CEC02
:105C400018F0420E8CEC18F0000E8CEC18F01200DC
:105C50007E0E8CEC18F0100E8CEC18F0080E8CEC0C
:105C600018F0140E8CEC18F0620E8CEC18F0120088
:105C70007E0E8CEC18F0400E8CEC18F0400E8CEC84
:105C800018F0400E8CEC18F0400E8CEC18F012005E
:105C90007E0E8CEC18F0040E8CEC18F0080E8CECD8
:105CA00018F0040E8CEC18F07E0E8CEC18F012003C
:105CB0007E0E8CEC18F0040E8CEC18F0180E8CECA8
:105CC00018F0200E8CEC18F07E0E8CEC18F0120000
:105CD0003C0E8CEC18F0420E8CEC18F0420E8CEC62
:105CE00018F0420E8CEC18F03C0E8CEC18F0120000
:105CF0007E0E8CEC18F0120E8CEC18F0120E8CEC60
:105D000018F0120E8CEC18F00C0E8CEC18F012003F
:105D10003C0E8CEC18F0420E8CEC18F0520E8CEC11
:105D200018F0220E8CEC18F05C0E8CEC18F01200BF
:105D30007E0E8CEC18F0120E8CEC18F0120E8CEC1F
:105D400018F0120E8CEC18F06C0E8CEC18F012009F
:105D5000440E8CEC18F04A0E8CEC18F04A0E8CECC9
:105D600018F04A0E8CEC18F0320E8CEC18F0120081
:105D7000020E8CEC18F0020E8CEC18F07E0E8CECFF
:105D800018F0020E8CEC18F0020E8CEC18F01200D9
:105D90003E0E8CEC18F0400E8CEC18F0400E8CECA3
:105DA00018F0400E8CEC18F03E0E8CEC18F012003F
:105DB000060E8CEC18F0180E8CEC18F0600E8CECC3
:105DC00018F0180E8CEC18F0060E8CEC18F012007F
:105DD0007E0E8CEC18F0200E8CEC18F0100E8CEC73
:105DE00018F0200E8CEC18F07E0E8CEC18F01200DF
:105DF000460E8CEC18F0280E8CEC18F0100E8CEC83
:105E000018F0280E8CEC18F0460E8CEC18F01200EE
:105E1000060E8CEC18F0080E8CEC18F0700E8CEC62
:105E200018F0080E8CEC18F0060E8CEC18F012002E
:105E3000620E8CEC18F0520E8CEC18F04A0E8CECC2
:105E400018F0460E8CEC18F0420E8CEC18F0120094
:105E5000440E8CEC18F0640E8CEC18F0540E8CECA4
:105E600018F04C0E8CEC18F0440E8CEC18F012006C
:105E7000300E8CEC18F0480E8CEC18F0480E8CECC0
:105E800018F0480E8CEC18F07E0E8CEC18F0120016
:105E9000CF0E8CEC18F0B70E8CEC18F0B70E8CEC23
:105EA00018F0B70E8CEC18F0810E8CEC18F0120084
:105EB000870E8CEC18F0EB0E8CEC18F0ED0E8CECE1
:105EC00018F0EB0E8CEC18F0870E8CEC18F012002A
:105ED000810E8CEC18F0B50E8CEC18F0B50E8CEC35
:105EE00018F0B50E8CEC18F0CB0E8CEC18F01200FC
:105EF000C30E8CEC18F0BD0E8CEC18F0BD0E8CECC3
:105F000018F0BD0E8CEC18F0DB0E8CEC18F01200C3
:105F1000810E8CEC18F0BD0E8CEC18F0BD0E8CECE4
:105F200018F0BD0E8CEC18F0C30E8CEC18F01200BB
:105F3000810E8CEC18F0B50E8CEC18F0B50E8CECD4
:105F400018F0B50E8CEC18F0BD0E8CEC18F01200A9
:105F5000810E8CEC18F0F50E8CEC18F0F50E8CEC34
:105F600018F0F50E8CEC18F0FD0E8CEC18F0120009
:105F7000C30E8CEC18F0BD0E8CEC18F0BD0E8CEC42
:105F800018F0AD0E8CEC18F0CB0E8CEC18F0120063
:105F9000810E8CEC18F0F70E8CEC18F0F70E8CECF0
:105FA00018F0F70E8CEC18F0810E8CEC18F0120043
:105FB000FF0E8CEC18F0BD0E8CEC18F0810E8CEC02
:105FC00018F0BD0E8CEC18F0FF0E8CEC18F01200DF
:105FD000CF0E8CEC18F0BF0E8CEC18F0BF0E8CECD2
:105FE00018F0BF0E8CEC18F0C10E8CEC18F01200FB
:105FF000810E8CEC18F0EF0E8CEC18F0F70E8CEC98
:1060000018F0EB0E8CEC18F09D0E8CEC18F01200D2
:10601000810E8CEC18F0BF0E8CEC18F0BF0E8CECDF
:1060200018F0BF0E8CEC18F0BF0E8CEC18F01200BC
:10603000810E8CEC18F0FB0E8CEC18F0F70E8CEC4B
:1060400018F0FB0E8CEC18F0810E8CEC18F012009E
:10605000810E8CEC18F0FB0E8CEC18F0E70E8CEC3B
:1060600018F0DF0E8CEC18F0810E8CEC18F012009A
:10607000C30E8CEC18F0BD0E8CEC18F0BD0E8CEC41
:1060800018F0BD0E8CEC18F0C30E8CEC18F012005A
:10609000810E8CEC18F0ED0E8CEC18F0ED0E8CEC03
:1060A00018F0ED0E8CEC18F0F30E8CEC18F01200DA
:1060B000C30E8CEC18F0BD0E8CEC18F0AD0E8CEC11
:1060C00018F0DD0E8CEC18F0A30E8CEC18F012001A
:1060D000810E8CEC18F0ED0E8CEC18F0ED0E8CECC3
:1060E00018F0ED0E8CEC18F0930E8CEC18F01200FA
:1060F000BB0E8CEC18F0B50E8CEC18F0B50E8CECD9
:1061000018F0B50E8CEC18F0CD0E8CEC18F01200D7
:10611000FD0E8CEC18F0FD0E8CEC18F0810E8CEC62
:1061200018F0FD0E8CEC18F0FD0E8CEC18F012003F
:10613000C10E8CEC18F0BF0E8CEC18F0BF0E8CEC7E
:1061400018F0BF0E8CEC18F0C10E8CEC18F0120099
:10615000F90E8CEC18F0E70E8CEC18F09F0E8CEC1E
:1061600018F0E70E8CEC18F0F90E8CEC18F0120019
:10617000810E8CEC18F0DF0E8CEC18F0EF0E8CEC2E
:1061800018F0DF0E8CEC18F0810E8CEC18F0120079
:10619000B90E8CEC18F0D70E8CEC18F0EF0E8CECDE
:1061A00018F0D70E8CEC18F0B90E8CEC18F0120029
:1061B000F90E8CEC18F0F70E8CEC18F08F0E8CECBE
:1061C00018F0F70E8CEC18F0F90E8CEC18F01200A9
:1061D0009D0E8CEC18F0AD0E8CEC18F0B50E8CEC1E
:1061E00018F0B90E8CEC18F0BD0E8CEC18F0120003
:1061F000000E8CEC18F0000E8CEC18F0040E8CECF9
:1062000018F00A0E8CEC18F0040E8CEC18F012004A
:10621000000E8CEC18F0000E8CEC18F0000E8CECDC
:1062200018F0000E8CEC18F0000E8CEC18F0120038
:10623000FF0E8CEC18F0FF0E8CEC18F0FF0E8CECBF
:1062400018F0FF0E8CEC18F0FF0E8CEC18F012001A
:10625000280E8CEC18F01200280E8CEC18F0280E8A
:106260008CEC18F0280E8CEC18F0280E8CEC18F042
:10627000280E8CEC18F01200100E8CEC18F0100E9A
:106280008CEC18F07C0E8CEC18F0100E8CEC18F0E6
:10629000100E8CEC18F01200100E8CEC18F0100E92
:1062A0008CEC18F0100E8CEC18F0100E8CEC18F032
:1062B000100E8CEC18F01200400E8CEC18F0200E32
:1062C0008CEC18F0100E8CEC18F0080E8CEC18F01A
:1062D000040E8CEC18F01200BF0E8CEC18F0DF0EE0
:1062E0008CEC18F0EF0E8CEC18F0F70E8CEC18F02C
:1062F000FB0E8CEC18F012007E0E8CEC18F07E0E6B
:106300008CEC18F0000E8CEC18F01200000E8CECE7
:1063100018F0000E8CEC18F0000E8CEC18F0120047
:10632000000E8CEC18F07E0E8CEC18F01200000EB3
:106330008CEC18F0000E8CEC18F01200000EAA6E17
:10634000000EA96E3F50FE0BA86EA69EA69CA684CA
:10635000550EA76EAA0EA76EA682A6B2ADEF31F0BB
:10636000A6941200000EAA6E010EA96E4F50A86EE0
:10637000A69EA69CA684550EA76EAA0EA76EA68200
:10638000A6B2C0EF31F0A6941200000EAA6E020E63
:10639000A96E5A50A86EA69EA69CA684550EA76EFE
:1063A000AA0EA76EA682A6B2D3EF31F0A694120071
:1063B000000EAA6E030EA96E2450A86EA69EA69C7F
:1063C000A684550EA76EAA0EA76EA682A6B2E6EF09
:1063D00031F0A6941200000EAA6E040EA96E25508C
:1063E000A86EA69EA69CA684550EA76EAA0EA76EA2
:1063F000A682A6B2F9EF31F0A6941200000EAA6EA2
:10640000050EA96E2650A86EA69EA69CA684550EC3
:10641000A76EAA0EA76EA682A6B20CEF32F0A694C3
:106420001200000EAA6E060EA96E2750A86EA69E38
:10643000A69CA684550EA76EAA0EA76EA682A6B22B
:106440001FEF32F0A6941200000EAA6E070EA96E7E
:106450005050A86EA69EA69CA684550EA76EAA0EA6
:0E646000A76EA682A6B232EF32F0A69412000A
:020000040030CA
:03000100381800AC
:02000500358044
:060008000FC00FE00F40E5
:0200000400F00A
:080000002000010000000000D7
:00000001FF
